:1000000040230020293100006D8B0000FD300000EE
:10001000FD300000FD300000FD3000000000000059
:10002000000000000000000000000000B52D0000EE
:10003000FD30000000000000612D0000FD300000D8
:10004000652E0000652E0000652E0000652E000064
:10005000652E0000652E0000652E0000652E000054
:10006000652E0000652E0000652E0000652E000044
:10007000652E0000652E0000652E0000652E000034
:10008000652E0000652E0000652E0000652E000024
:10009000652E0000652E0000652E0000652E000014
:1000A000652E0000652E0000652E0000652E000004
:1000B000652E0000652E0000652E0000652E0000F4
:1000C000652E0000652E0000652E0000652E0000E4
:1000D000652E0000652E0000652E0000652E0000D4
:1000E000652E0000652E0000652E0000652E0000C4
:1000F000652E0000652E0000652E0000652E0000B4
:1001000053B94AB9002908BF00281CBF4FF0FF317E
:100110004FF0FF3000F00CB8ADF1080C6DE904CEE3
:1001200000F008F8DDF804E0DDE9022304B07047D0
:10013000704700BF2DE9F04786468C460846089E6A
:10014000154674461946002B40F0C2808542B2FA2B
:1001500082F245D94AB1C2F1200300FA02FC2EFA1C
:1001600003F3954043EA0C0C94404FEA154EA8B2B5
:10017000BCFBFEF8230C0EFB18CC08FB00F943EA8D
:100180000C43994528D9EB1808F1FF3704D299455B
:1001900002D9A8F102072B44A3EB0903A4B2B3FBD5
:1001A000FEFC0EFB1C330CFB00F044EA0344A042AF
:1001B00014D92C190CF1FF3304D2A04202D9ACF1AE
:1001C00002032C44241A43EA07401EB1D440002302
:1001D00034607360BDE8F0874746DDE76346F1E7CA
:1001E00092BB431B01214FEA154EAFB2B3FBFEFC9D
:1001F000200C0EFB1C330CFB07F840EA0343984528
:1002000062D9EB180CF1FF3004D2984502D9ACF159
:1002100002002B44A3EB0803A4B2B3FBFEFC0EFBCD
:100220001C330CFB07F744EA0344A7424ED92C19B0
:100230000CF1FF3304D2A74202D9ACF102032C44E3
:10024000E41B43EA0040C0E7C2F1200320FA03F1B7
:10025000954090402EFA03F303434FEA154EAFB298
:10026000B1FBFEFC0EFB1C10190C0CFB07F841EA5D
:100270000041884504FA02F422D969180CF1FF30D4
:1002800004D2884502D9ACF102002944A1EB08014F
:100290009BB2B1FBFEFC0EFB1C110CFB07F743EA03
:1002A00001439F420ED9EB180CF1FF3104D29F425B
:1002B00002D9ACF102012B44DB1B41EA004192E779
:1002C0006046E3E76146F7E76046A3E76346B7E7C2
:1002D000834206D916B9002108467BE7C6E900E04B
:1002E000F9E7B3FA83F78FB9834201D3724508D88F
:1002F000BEEB020460EB030301209C461EB9002103
:1003000068E73846FAE7C6E9004CF8E7C7F1200C81
:10031000BB4022FA0CF41C432EFA0CF120FA0CF329
:10032000B84001434FEA14490EFA07F5B3FBF9F858
:100330001FFA84FE09FB18300B0C08FB0EFA43EA87
:1003400000439A4502FA07F240D9E31808F1FF305A
:1003500004D29A4502D9A8F102002344A3EB0A0370
:1003600089B2B3FBF9F809FB183308FB0EFE41EA2A
:1003700003418E452CD9611808F1FF3304D28E4514
:1003800002D9A8F10203214443EA0040A0FB0298ED
:10039000A1EB0E014145CE46434602D306D14D4561
:1003A00004D2B9EB020E68EB04030138002EA6D08C
:1003B000B5EB0E0261EB030101FA0CFC22FA07F324
:1003C0004CEA0303F940C6E9003198E74046C5E727
:1003D0004346D9E7014B1B681B68184758080020A3
:1003E000014B1B685B68184758080020014B1B68CD
:1003F0009B68184758080020014B1B68DB681847AA
:1004000058080020014B1B681B691847580800203A
:10041000014B1B685B69184758080020014B1B689B
:100420009B69184758080020014B1B68DB69184777
:1004300058080020014B1B681B6A18475808002009
:1004400018B1034B1860002070476FF0150070471B
:10045000580800202DE9F041046803792769012537
:100460009D4063681B681D420E460AD11449154819
:1004700040F2924208F05EFB114840F2924108F0CF
:1004800052FB3B681D4263681B6818BF86F001067B
:100490001D420AD10A490B484FF48D6208F04AFB0D
:1004A00007484FF48D6108F03EFB36B1A368DB6866
:1004B00029462046BDE8F0411847A3681B69F7E7C5
:1004C000FE9B00002F9C0000072810B504460AD9A7
:1004D0000749084840F27D2208F02CFB044840F20E
:1004E0007D2108F020FBA000303000F0FC0010BDA2
:1004F000479C00002F9C0000072810B504460AD92D
:100500000749084840F2852208F014FB044840F2ED
:10051000852108F008FBA000603000F0FC0010BD51
:10052000479C00002F9C00002DE9F8439846384B6B
:1005300000289146A3F1080206460D460CBF13465B
:100540000426A2F11C07B9F1000F39D097F84D40ED
:1005500018795B794B4536D0FFF7CEFF00F180402C
:10056000012101FA04FE00F5C040E400B9F1000FDA
:1005700041D0D7F850C00023CCF84031DCF84031EE
:10058000CCF84085DCF8002242F480720A43CCF8B3
:10059000002204F1804202F5F8320CF5A073C2F893
:1005A0001035C2F814051B4806F18043C0F804E575
:1005B00065B903F58053CCF800101960BDE8F883E5
:1005C00097F84E40C4E7FFF77FFFC7E797F84C4026
:1005D000E20002F1804202F5F83203F58053C2F8DE
:1005E0001055C2F814C504F51172A14040F822302C
:1005F000C0F80415E2E704F1804303F5F833C3F8CB
:100600001055C3F81405034BC3F804E5D6E700BF43
:100610002400002000F0014038B5144BBFF35B8F7D
:100620001446022253E8005F012D04D143E8002C58
:10063000BCF1000FF6D1BFF35B8F13D10C4B0D4D06
:10064000186029602346014601220020FFF76CFF55
:10065000296809B9002038BD002223461046FFF75B
:1006600063FFF7E76FF00F00F5E700BF5C080020BD
:10067000640800206008002008B5094B98420BD0A0
:10068000084B98420AD008490848DD2208F052FA7F
:100690000548DD2108F047FA002008BD0120FCE7ED
:1006A000D8960000C09600007C9C00002F9C0000A3
:1006B00008B5074B0246D3F8500600F001001AB106
:1006C00008F031F90B3808BD08F011F9FAE700BF5E
:1006D000001000402DE9F041184BBFF35B8F154629
:1006E00006460F46022253E8001F012903D143E8C2
:1006F00000200028F7D1BFF35B8F1CD110480121E7
:10070000FFF7A8FE044698B90E4BDFF83C801E6048
:10071000012231462B461046C8F80070FFF704FF4F
:10072000D8F8001021B12B4622460120FFF7FCFE2D
:100730002046BDE8F0816FF00F04F9E75C08002067
:100740001000002064080020600800202DE9F14F0F
:1007500005680679B0F806B00BF03003302BD5E908
:1007600001A82F690AD1224922484FF42E7208F0BD
:10077000E1F91F484FF42E7108F0D5F90BF006038C
:10078000042B0AD11A491B484FF4307208F0D2F9F1
:1007900017484FF4307108F0C6F9DAF80030012438
:1007A0001BF0010F04FA06F40CBF4BF4B01B8BF4E2
:1007B000D01B1C422BF480190AD10D490D484FF46F
:1007C000357208F0B7F90A484FF4357108F0ABF903
:1007D0003B681BF0010F14BF2343A3433B60D8F8D1
:1007E00000304A463146284601B0BDE8F04F184770
:1007F000FE9B00002F9C0000064BBFF35B8F014661
:1008000053E8000F43E80012002AF9D1BFF35B8FD1
:10081000704700BF5C08002010B5144BBFF35B8F1E
:10082000022253E8001F002903D143E800200028DA
:10083000F7D1BFF35B8F15D10D480121FFF70AFEF9
:10084000044640B901460B48FFF704FE044610B9C0
:10085000122008F0E5FEB4FA84F04009FFF7CCFF5F
:10086000204610BD6FF00F04FAE700BF5C080020BF
:100870003C0000201000002010B50F4BBFF35B8F31
:10088000022253E8001F012903D143E80020002879
:10089000F7D1BFF35B8F0BD108480021FFF7DAFDDA
:1008A0000446003818BF0120FFF7A6FF204610BD00
:1008B0006FF00F04FAE700BF5C0800203C00002046
:1008C000F0B5214BBFF35B8F87B00546022753E895
:1008D000002F012A03D143E800710029F7D1BFF3AB
:1008E0005B8F2DD11F2D28D8184E00213046FFF7E1
:1008F000B1FD0446D8B9C0238DF8043001ABCDE971
:100900000237012102ABBD4030468DF805500493FB
:100910000591FFF79FFD044648B956F8100C83680F
:1009200004AA1D68A6F10C012346A847044601202D
:10093000FFF762FF204607B0F0BD6FF01504F6E741
:100940006FF00F04F6E700BF5C08002010000020E5
:100950002DE9F041314CDFF8C88094F84D50012763
:1009600007FA05F3ED0005F1804505F5F835C8F8FF
:1009700008350026C5F8106594F82000FFF7A4FD9F
:10098000C5F8146594F84D5094F82800A23508EB8A
:10099000C505FFF799FD234B6E601B68B3B194F852
:1009A0004C309F40DA009B0002F1804203F180430B
:1009B00002F5F83203F5F833C8F80875C2F8106587
:1009C000C2F81465C3F81069C3F81069164B1B68A8
:1009D000F3B194F84E50124E0123AB40ED0005F1F7
:1009E000804505F5F835C6F808350027C5F81075B7
:1009F00094F82000FFF780FDC5F8147594F84E5068
:100A000094F82800A23506EBC506FFF775FD776060
:100A1000BDE8F0410120FFF7EFBE00BF000000205D
:100A200000F00140640800206008002038B504464A
:100A30000220FFF7E1FE022805460FD044B1012C49
:100A400006D06FF015042846FFF7D6FE204638BDC5
:100A500021460448FFF7FEFC0446F4E76FF00F045C
:100A6000F4E700BF44000020154890F8283090F8C3
:100A700029109B0003F1804303F5C04381F001017D
:100A8000D3F8102522F4801242EA0152C3F810254F
:100A900090F8203090F821109B0003F1804303F57B
:100AA000C04381F00101D3F8102522F4801242EAFC
:100AB0000152C3F8102500211030FFF7CBBC00BF56
:100AC00000000020F8B5634C236DE06BD3F80425DB
:100AD00022F00302C3F80425D3F8082522F003020C
:100AE000C3F80825D3F8102522F00F0242F00402C3
:100AF000C3F8102508F032FD10B96FF01200F8BDF0
:100B000004F13C00FFF722FE0028F8D1606C08F0E9
:100B100025FD0028F1D004F14400FFF717FE00285E
:100B2000EDD104F1200004F0E9FD4B4B984206465C
:100B300002D06FF00500E2E7E06AFFF79DFD94F850
:100B4000303003F01F0343EA4013012704F128006B
:100B5000E36184F8217004F0D1FDB0420546E8D18C
:100B6000606BFFF789FD94F8203094F8382094F8F2
:100B7000216084F829709B0003F1804303F5C04392
:100B800002F01F0242EA40127E403448D3F810754A
:100B9000E16962620740C3F81075D3F81075090265
:100BA00001F47C51394341EA0651C3F81015D3F8DA
:100BB000101541F00301C3F8101594F828309B007C
:100BC00003F1804303F5C0431202D3F8101501402E
:100BD000C3F81015D3F8101502F47C520A43C3F879
:100BE0001025D3F8102542F00302C3F8102504F1B4
:100BF0004D0004F021FFA84206469AD104F14E00B0
:100C000004F01AFFB042054693D104F14C0004F001
:100C100013FFA8428DD1206908F0A0FC00283FF402
:100C20006CAF0F4C2046FFF791FD00287FF467AFB3
:100C30000C4805F07FFD44F8100C00283FF479AF14
:100C400008F08CFC00283FF458AFBDE8F840064897
:100C5000FFF7F6BB000000200000AD0BFFC0ECFF6B
:100C600010000020A09C0000089900002DE9F74F1B
:100C7000424807F08FFE0026414808F06FFC10B98B
:100C8000404807F087FE00F09BFB014610B13E484C
:100C900007F080FE3A4FDFF8F4B04FF0000800F0A4
:100CA00051FCD7F80890D9F800305BB10DF105017F
:100CB00038469847014640B1431CF0D0344807F00D
:100CC00069FEECE76FF05701F8E7B8F1000F11D1BA
:100CD0009DF80560360208F0A1FC4FF47A73A0FB82
:100CE000030503FB0155C40B44EA45444FF00108DA
:100CF000ED0BD4E708F092FC4FF47A7AA0FB0A03DC
:100D00000AFB0131C30B43EA41431B1B4FEAD131BC
:100D100061EB0501062B71F100019DF805300BDB3D
:100D20001E0208F07BFCA0FB0A050AFB0155C40B60
:100D300044EA4544ED0BB2E71E433146584607F0FE
:100D400029FE304600F018FC0DF1060000F066FEAA
:100D500088B1BDF806100F4807F01CFEBDF806105C
:100D6000090AD9F80430384698479DF80610D9F892
:100D70000430384698474FF0000890E7A69C0000E2
:100D800008970000C99C0000E09C00001D9D000029
:100D9000059D0000399D0000084B0022C3F81C216E
:100DA000D3F81C2101225A61D3F81C21002AFBD060
:100DB000D3F8480500F07F00704700BF00100040E6
:100DC000124AD8B1D2F83C3723F0004323F0FF0396
:100DD00043F0004343F07D03C2F83C37D2F87C3740
:100DE00023F0004323F0700343F0004343F060031B
:100DF000C2F87C37064B83F84D027047054BC2F8AA
:100E00003C37D2F87C3723F00043F1E70010004074
:100E1000580000203430004070B5114D114995F84C
:100E20006434114C012202FA03F3C1F8083500239F
:100E3000C4F80032C4F81031D4F810312261D4F86B
:100E40001031002BFBD00026C4F810610120D4F82B
:100E5000103101F001FF0B23C4F80833EE8070BDA0
:100E60005800002000F001400010004038B5104C40
:100E7000104A94F86434012505FA03F1DB0003F10C
:100E8000804303F5F833C2F808150022C3F8102593
:100E900004F51170C3F8142505F078FBFFF7BCFFCB
:100EA000FFF7B0FAFFF7B4FAFFF79AFA257038BDEA
:100EB0005800002000F00140044B0548D3F84432AC
:100EC000D3F81035DBB2D840704700BF580000207F
:100ED0000071020010B5064C204605F057FB204675
:100EE00005F098FB04F10800BDE8104006F0AEB82C
:100EF000840200201FB5304C94F84E1294F84F0233
:100F000000F096FD40B92D4807F044FD01236380B1
:100F10006FF0150004B010BDFFF77EFF284B94F86A
:100F20004F22C3F80C2594F84E22C3F81025D4F8AC
:100F30002022110E1202C3F82415C3F81C25012229
:100F4000C3F8302500211F4AC3F82C15C3F83C25EF
:100F500040F20312C3F8342540F25B62C3F838252F
:100F600068460D2207F04AFE94F84E329DF80310B1
:100F700094F81C22033B012B81BF03238DF807301B
:100F800002238DF804309DF807305B0743EA0153D4
:100F90009DF8041043EA815343EA02639DF806205A
:100FA00043EA8263064A43F48473C2F81435064B5D
:100FB000C2F818350020ADE758000020549D00000D
:100FC0000010004055555500FF0003006D4BD3F84D
:100FD00004212DE9F0417AB16B480022C3F80421C5
:100FE000D3F804310378042B06D190F84C321BB1AE
:100FF00000F5117005F0CAFA624AD2F80C31002BE4
:1010000000F094800025C2F80C51D2F80C315F4BEF
:101010005D4C0221C3F880112378042B40F08680B8
:10102000D4F80C6204F10803F11A4B424B414FF41F
:10103000817101FB03430833C4F80C32C2F8043554
:10104000FFF7E0F9FFF7E4F9D4F8582450492846AF
:10105000FFF7D2F994F84C323BB3FFF72DFF294646
:101060000246012304F5117008F045FA4FF4FA71B5
:10107000D4F8440207F05DFC01230246194604F54A
:10108000117008F038FAD4F84432C3F84051D3F85C
:101090004021C3F8445104F51170D3F8443105F0F0
:1010A000B9FA04F5117005F04DFA364BD3F8003457
:1010B000DB0735D594F8503294F84E0235787778BE
:1010C000002BA0F103030CBF4FF002084FF0030800
:1010D000012B05F00F0513D8022D21D807F03BFC9A
:1010E000A5B1022D47D15522711C0023D8B28742E9
:1010F00013D911F8010F904203F10103F6D00FE06C
:1011000007F029FC08B1042D0AD875BB21493A46DD
:1011100006EB080007F057FD10B9E3880133E380C0
:101120004FF481720021304607F068FD154BD3F86B
:10113000002122B3144C0022C3F80021D3F800315F
:101140002378042B1BD194F84C32C3B104F51170F1
:1011500005F060FA04F5117005F03AFA78B904F573
:101160001170BDE8F04105F0EDB9022DBBD0042DA2
:1011700003D0012DD4D10F22B6E7FF22B4E7BDE89A
:10118000F08100BF001000405800002000E100E0A6
:10119000101100406C9E000070B5404DD5F818420B
:1011A000640004F66214A4B240F6C4139C420646DE
:1011B0000DD93B493B484FF4BF6207F0BBFC3848B0
:1011C0004FF4BF6107F0AFFCA4F5166412E040F6DF
:1011D00037139C4248D83249324840F2FB5207F05C
:1011E000A9FC2F4840F2FB5107F09DFCA4F63814EF
:1011F00044F480742C4BD5F80C22C3F80845C3F88E
:1012000004250022C3F80021D3F800210322C3F8EB
:101210000022D5F85C0420B995F84E123046FFF74D
:1012200003F9224BC5F858040222C3F8802101209B
:1012300001F004FD1C490B23C1F8043395F84C322E
:10124000B6B113B10120FFF7BBFD0024C1F80C417A
:10125000D1F80C31FFF7BEF8D5F8582414492046D0
:10126000BDE87040FFF7C8B8B4F5166FACD2BDE763
:1012700095F84F22C1F80C257BB10E4805F086F990
:101280000C4805F0C7F9D5F84432C3F84061D3F8EB
:101290004021C3F84461D3F8443170BD58000020A8
:1012A000849D00002F9C00000010004000E100E041
:1012B000101100409C020020B0F5A07F38B503D08B
:1012C000B0F5A27F45D038BD394DFFF765FD95F8E3
:1012D0004D327BB35F2802D90020FFF771FD354BFB
:1012E000354801241C649C6305F050F9FFF7E4FDC8
:1012F000002102462346304808F0FDF82E4805F04C
:1013000089F9D5F844322C480022C3F84021D3F89B
:10131000403105F017F9D5F8442242F30732002A8C
:10132000D1DB530902F01F0294406033234A42F894
:101330002340C8E71F4BD3F874354FF6F0721342C1
:1013400003D15E28CBD80120C7E7B3F5003FF8D220
:10135000F9E7174DFFF720FD95F84D321BB35E28D6
:1013600002D90020FFF72CFD124BD5F84422124879
:1013700001241C649C630023C2F84431D2F8442148
:1013800021461A4608F0B7F8D5F8443243F307333C
:10139000002B98DB5A0903F01F039C406032074B77
:1013A00043F822408FE75E28DED80120DAE700BF4D
:1013B00058000020001000409C02002000E100E0E6
:1013C000F0B5002087B002F0D3F938B9524807F0E1
:1013D000E1FA6FF00504204607B0F0BD0023039347
:1013E000059302A90123049300F07CFD041E04DA96
:1013F0004A48214607F0CEFAEDE7049B9B07FCD153
:10140000059C14B146482146F4E7464A464804275D
:1014100002A9CDE902448DF8087005F001F8434BAC
:101420009842064601D0314625E0414D224603212F
:10143000082001F033FC40F27121D5F8240207F0B6
:1014400078FA01230246214605F50970009408F058
:1014500068F805F5097005F075F8364A02A905F532
:101460000B70CDE902448DF8087004F0D9FFB0424A
:10147000074606D00146304807F08CFA6FF00A04A0
:10148000A9E722460321092001F008FC4FF48271EC
:10149000D5F82C0207F04DFA01230246214605F546
:1014A0000B7008F028F80723244A02A905F51170EB
:1014B000CDE902448DF8083004F0B2FFB842064688
:1014C000B1D1224602211A2001F0E8FBFFF7F4FC1B
:1014D00021460246012305F5117008F00CF805F2CB
:1014E000644004F0A9FAB042014601D01448C3E7B1
:1014F00022460221012001F0D1FB012001F09EFBD8
:10150000FFF7F8FC044600287FF465AF01232B7039
:101510002871C5F810025EE7B89D0000D99D000053
:10152000F39D0000318900007C0200200000AD0B1B
:1015300058000020D50E0000139E0000B9120000D4
:10154000349E000008B5094804F0FCFF08484FF03D
:10155000FF324FF0FF3305F0AFFD014620B1BDE88B
:101560000840044807F016BA08BD00BF84020020F6
:101570008C020020589E00002DE9F0419F4C012371
:1015800023710023638023780646870B4FEA1028D7
:10159000C5B2002B00F03382002F40F01D81FFF711
:1015A00065FCB8F1090F00F28D80DFE818F00A0041
:1015B0002900310089008F00940010018B008B00FE
:1015C000A600032D7ED88E4A00250323C4F81052AE
:1015D00084F84E3284F81C52D2F8403723F000438E
:1015E000C2F840372846FFF7EBFB864804F0CEFFF1
:1015F00084F84C52FFF77EFC00231846BDE8F081CA
:101600000F2D5FD82D0105F0C005C4F81052F3E787
:10161000043D0F2D56D8DFE805F008080808212101
:1016200021213838383851515151754A002503234A
:1016300084F84E3284F81C52D2F8403723F000432D
:10164000C2F840372846FFF7BBFB6E4804F09EFF08
:1016500084F84C52FFF74EFCC3B2CEE70423684A2D
:1016600084F84E32012384F81C32D2F8403723F03C
:101670000043C2F840370020FFF7A2FB614804F0A6
:1016800085FF002384F84C32E4E7052384F84E32CA
:101690005B4A032384F81C32D2F8403723F000431E
:1016A00023F47F4343F0004343F44443C2F84037FC
:1016B000D2F88837002BCDD10123E3E70623E5E7F5
:1016C000032D99D901236380042396E7032DF9D8CC
:1016D0001623638090E70F2DF4D8DFE805F00808A3
:1016E00008080B0B0B0B080808080B0B0B0B4FF42F
:1016F000FF73EEE744F29023EBE707F036F98046FC
:1017000000F0A8F976B27E2E074608D107F029F935
:10171000C0B284F84F02400040F4007009E07F2E10
:101720000AD107F020F9C0B284F84F02400040F41B
:101730008060608000208FE77F35EDB2932D19D94E
:1017400094F84F526B0043F00103638007F009F9EE
:10175000854205D1638843F40073638004207BE7EE
:1017600094F84F5207F0FFF88542F7D1638843F4AD
:101770008063F2E707F0F5F840B28642C6DD07F075
:10178000F2F840B28642CCDA012300E001339845FA
:1017900019D957F823506AB29642F7DA03F1804319
:1017A000013B921B57F823104BB2002AA3EB060310
:1017B000B8BF5242002B52B2B8BF5B429A42B8BF88
:1017C000294684F84F1294F84F024000B1E70DB15A
:1017D0000123C2E728463FE7032F15D1012B03D190
:1017E00001236380022308E7E3886FEA43436FEA3B
:1017F00053436380FFF73AFBFEE600BF580000202A
:10180000001000409C020020012BE9D1D4F81022E6
:1018100005F00305C6F3850602F0C00208F03F009C
:101820003243032DC4E98425C4F8180203D02728C5
:101830000AD96380E1E694F84E32033B012B94BF52
:10184000FE23FF23C4F81432DFF8B8C1C4F80CC279
:101850000021012FE1800AD14FF40172604607F0A8
:10186000CDF93846FFF798FC04232370C4E6D4F87A
:10187000141294F85032FE29D5B262D0002B0CBF5E
:10188000022303230229657258D049D800294DD17B
:1018900021720CEB03005C4907F0A5F994F8503273
:1018A00043B1D4F80C321A7842F020021A7094F83E
:1018B00056249A700020FFF76FFC94F84E22D4F85B
:1018C0001032062A40F28880DB0094F8501221B1D1
:1018D00094F8541402EBC102134440F27121F9331D
:1018E0000A46934201F27121FAD80023474819466B
:1018F00007F001FEFEF76EFDD4F86004FF2804D067
:10190000FEF78CFD00287FF4DDAED4F82402D4F875
:1019100058243F4900F5A070FEF768FD0223A4E7B4
:10192000FF297FF4CFAE0420207202E00121217252
:101930000F210CEB030007F061F9AFE7217255218D
:10194000F7E76572062E3FF657AEDFE806F00404AF
:10195000223F333639000020FFF71EFC2D4B4FF499
:101960000072C3F850260122C3F80022FEF732FDB0
:10197000D4F86004FF2804D0FEF750FD00287FF45F
:10198000A1AED4F8582422490020FEF72FFD0323EE
:101990006BE7C5B218F0300F18BF45F0C00594F8DA
:1019A0004E12284600F044F800283FF48BAE84F82D
:1019B0004F5221E6C4F860041EE6C4F85C041BE63E
:1019C000FF230020C4F86034C4F85C04FEF732FD45
:1019D00000283FF411AE75E60F49052A31F81210C0
:1019E00002D101EB831370E7062A02D101EB031346
:1019F0006BE701EBC303042A08BF5B0865E7052317
:101A0000FBE500BF600000206C9E00007C0200200F
:101A10001011004000100040F09B0000034B00211B
:101A20001A7919715B8803801046704758000020AE
:101A30000339032908D8064A002352F8041B8842B8
:101A400004D001330F2BF8D10020704701207047DC
:101A50002C990000004870472C990000436803F05F
:101A60000303032B10B50446816002D02BB1002084
:101A700000E000680023636010BD05490548452269
:101A800007F058F80248452107F04DF8EFE700BF8E
:101A90006B9F00002F9C00000B6801330B60014B13
:101AA0001B681847C004002007B50B4600210246FA
:101AB0000191034801A900F09BFA03B05DF804FB13
:101AC000991A00002DE9F84F858B2B07044617461D
:101AD00062D4022905F0070500F0C481AA46D4F8B3
:101AE0001890A38BB9F1000F71DA0022D4F80080AE
:101AF00023F00703C4E9002243F00103A383A38B6F
:101B000003F0070555454FF0000640F07D814FF08A
:101B1000000AB8F1000F00F0E18043F0080304F17F
:101B2000140BA383584605F0E1F840B9B049B14819
:101B3000B92206F0FFFFAE48B92106F0F4FF87F3A3
:101B40001188BFF36F8FBAF1000F40F06481B8F1D4
:101B5000000F40F0758116B1A7492046B0474FF0FD
:101B60002003EFF3118783F31288BFF36F8F58467A
:101B700005F0AEF840B99E499E488E2206F0DAFF85
:101B80009B488E2106F0CFFF584605F0BFF8A38B87
:101B900023F00803A38356E001290CBF45F010058C
:101BA00045F02005858304F1140005F09FF840B945
:101BB0008F499048B92206F0BDFF8D48B92106F043
:101BC000B2FF87F31188BFF36F8FBDE8F88F03F082
:101BD0000702511F012921D80021062AD4F80080CC
:101BE000C4E9001116D1424603E0E18B12680131CD
:101BF000E183002AF9D123F0070343F00202A28314
:101C0000204606F0D4FE00283FF479AF42F02002CF
:101C1000A28374E723F007039AB2F0E7042A1ED1E7
:101C200023F007039AB2A283204606F0C0FE10B14B
:101C300042F02002A283A38B03F00705002655453E
:101C4000B04640F0E180B4F81CA01AF0100F00F08C
:101C500000812AF01003A3830AF0070A3FE76749CF
:101C6000644840F21B1206F065FF644840F21B1105
:101C700006F059FFDFE755B160495E484FF4AB729B
:101C800006F058FF5D484FF4AB7106F04CFF236837
:101C900053B95A49574840F2571206F04BFF57487C
:101CA00040F2571106F03FFF23691E6856B95349A9
:101CB00050484FF4AD7206F03DFF50484FF4AD71FF
:101CC00006F031FFA38B23F0070343F006039BB21A
:101CD000062DA38340F094804FF000094FF0000AD6
:101CE000D046002E7FF419AFADE7022D0AD043494C
:101CF000404840F25D1206F01DFF404840F25D1181
:101D000006F011FFE38B53B13C493A484FF4AF72F0
:101D100006F010FF39484FF4AF7106F004FF236955
:101D20005E6856B93549334840F2611206F002FF49
:101D3000324840F2611106F0F6FEA38B23F0070350
:101D400043F004039BB2042DA383C5D04FF00008D9
:101D5000C146042558E0012D0AD0284925484FF4F2
:101D6000B27206F0E7FE25484FF4B27106F0DBFED2
:101D7000236853B921491F4840F2651206F0DAFE84
:101D80001E4840F2651106F0CEFE23699E6856B9E2
:101D90001A4918484FF4B47206F0CCFE17484FF4B5
:101DA000B47106F0C0FEA38B23F0070343F00503D4
:101DB0009BB2052DA3838FD04FF00008C1460525A7
:101DC00022E040F26B120D490A4806F0B3FE0B48C0
:101DD00040F26B1106F0A7FEA38B03F00702AA42A4
:101DE0003FF431AF4FF0000815464646C1460BE0C0
:101DF000B09F00002F9C0000911E00008E9F0000ED
:101E00004FF00008C1460625A268002A3FF47FAEC5
:101E10004FF0010A81E6A16800293FF498AE0F68EF
:101E200000293FF494AED1F804A04B462A46204640
:101E3000D0471FB13B6839461F46F1E73B46FAE7FA
:101E400041464B462A462046D8F8008006F0DBFD86
:101E50007DE61AF0200F3FF4A6AE2AF02003A383FC
:101E60000AF00705204606F0A2FD00283FF49BAECD
:101E700001380428A5D801A353F820F0DD1A00008A
:101E8000C31D0000771C0000EB1C0000571D000064
:101E9000F8B504460D4600F114064FF02003EFF3A9
:101EA000118783F31288BFF36F8F304604F010FF61
:101EB00040B90A490A488E2206F03CFE07488E21A6
:101EC00006F031FE304604F021FFA5613A46204677
:101ED0000121BDE8F840FFF7F5BD00BFB09F00004D
:101EE0002F9C00002DE9F04704460F4606F07BFDCD
:101EF000051E6DDB04F114094FF02003EFF3118A86
:101F000083F31288BFF36F8F484604F0E1FE40B9B7
:101F1000344935488E2206F00DFE32488E2106F0F7
:101F200002FE484604F0F2FEE38BA68B4FF6FF72EA
:101F3000934206F007064ED0022E1FD10133E383F1
:101F400035464FF00108484604F0D0FE40B9254917
:101F50002548B92206F0EEFD2248B92106F0E3FD3E
:101F60008AF31188BFF36F8FB8F1000F30D00023D0
:101F700032463946204606F046FD29E0062E0ED8A8
:101F8000DFE806F004180D0D042C040000233B606C
:101F90006368A3B9C4E90077A6B135460CE01349DC
:101FA000114840F2C91206F0C5FD104840F2C911AF
:101FB00006F0B9FD6FF004054FF00008C3E71F609D
:101FC0006760E9E7524602212046FFF77BFD354670
:101FD0002846BDE8F0876FF00A05EDE76FF085054C
:101FE000EAE700BFB09F00002F9C00008E9F00001A
:101FF0002DE9F04F814695B08B4617461C460025CB
:10200000387808B9284658E37B1C2528039306D066
:102010005946C8470028C0F25083013504E218220F
:1020200000210EA806F0EAFD7B78252B7DD0002349
:10203000781C98469E469C461E46014610F8012B89
:102040002B2A00F0A18000F29880202A00F09F80C7
:10205000232A00F09F802BB19DF8403043F04003CD
:102060008DF84030B8F1000F05D09DF8403043F0B6
:1020700020038DF84030BEF1000F05D09DF84030B0
:1020800043F010038DF84030BCF1000F05D09DF8EF
:10209000403043F008038DF840302EB19DF84030B9
:1020A00043F004038DF840309DF8403003F04400C5
:1020B000442803D16FF386138DF840309DF84030EB
:1020C0002A2A43F080038DF840307FD19DF84120CB
:1020D00042F001024B1C8DF841201A782E2A9DF8FF
:1020E00041200CBF0121002161F341028DF8412004
:1020F00078D15A782A2A6ED0013300224FF00A0C88
:10210000194611F8010BA0F13006092E40F2958016
:102110009DF840101292C1F3400040EAD2700A4686
:1021200060F341028DF840205CE0BA1C03928DF808
:1021300043309DF84130DA0740F12E8154F8048B8A
:10214000B8F1000F07DA9DF8402042F004028DF844
:102150004020C8F100085E0740F1278154F804AB25
:10216000BAF1000F80F226819DF841306FF34103F0
:102170008DF841304FF0FF3A1CE12D2A0DD0302A66
:102180007FF469AF012358E74FF0010C55E74FF09A
:10219000010E52E74FF001084FE701264DE70EFB15
:1021A0000262303A0346184610F8016BA6F1300C73
:1021B000BCF1090FF3D999428FD09DF840101192CC
:1021C000D20F62F341018DF8401086E70B460022E2
:1021D0004FF00A0EE7E79DF8412042F004028DF827
:1021E000412002331A786C2A47D02BD8682A31D084
:1021F0006A2A4BD04C2A51D01A4612F8013B03925E
:10220000782B9DF841208DF8433000F2BE806D2B75
:1022100051D8692B00F2B980572B67D8412B03D0D6
:10222000453B022B00F2B1809DF84230042262F35C
:1022300002038DF84230012373E00CFB0202303AB6
:102240000B465DE7742A25D07A2AD5D19DF8412026
:1022500006210CE05A78682A9DF8412006D1012118
:1022600061F3C6028DF841200233C5E7022161F314
:10227000C6028DF841200133BEE75A786C2A9DF8DA
:10228000412001D10421EBE70321F0E79DF8412033
:102290000521ECE79DF841200721E8E7BDF8402043
:1022A00022F4F04222F0020242F4804242F00202A2
:1022B000ADF84020DFE76E3BD9B201238B4040F2FE
:1022C00082410B4237D113F0240F51D1D8075CD58E
:1022D0009DF84230032161F302038DF8423002F091
:1022E0007803A3F140014B424B411AE0A3F158019E
:1022F000C9B2012000FA01F111F4624F94D140F605
:10230000010631421DD111F4043F3ED09DF8423008
:1023100060F3020302F07802402A8DF8423034D094
:1023200000239DF84020C2F340010B4363F34102B8
:102330008DF84020FDE69DF84230022161F3020352
:10234000E8E79DF84210022002F0780260F30201F3
:10235000402A8DF8421002BF9DF8401041F0010163
:102360008DF84010632BDBD1131E18BF0123D8E773
:102370009DF84230032161F3020312F0780F8DF8CB
:10238000423014BF01230023CBE79DF8403043F0D7
:1023900001038DF84030C3E79DF94020002AB4BF07
:1023A000DDF844804FF0FF38D5E698077FF5E2AEC0
:1023B000DDF848A09DF841100023CDE911339DF8C8
:1023C000423003F00703012BC1F3C30133D1CB1E0D
:1023D000042B04D8DFE803F01046461010002368F1
:1023E00001294FEAE372CDE90E320BD103F0FF036E
:1023F0000E9300230F9307E054F8043BDA17CDE95E
:102400000E3202E0022911D004349DF8403013F05E
:10241000030647D0039B3A465946484606F06CFBF4
:102420000028C0F24A810544039FE9E51AB20E92E2
:1024300043F3C033DEE7022B24D1CB1E042B04D898
:10244000DFE803F0181010181800012954F8043BB5
:102450004FF0000214D00229CDE90E32D5D19BB243
:102460000E93D2E7073424F00704F4E80223CDE901
:102470000E23CAE754F8043B0E9300230F93C4E7DE
:10248000DBB2BCE7042B08D1073424F00704D4E9FD
:1024900000230834CDE90E23B7E7032BB5D154F858
:1024A000043BDDE79DF843007828BDD862281CD89E
:1024B00025283FF4ADAD5828B6D10DF13603009371
:1024C000DDE90E0108AB10AA06F0D0FABAF1000F50
:1024D000074680F29A80002FA6D00DF13603D81B54
:1024E000002E00F0C1800130BEE0633815289BD873
:1024F00001A252F820F000BFCD250000DF2500002A
:102500002924000029240000292400002924000097
:10251000DF250000292400002924000029240000D0
:10252000292400006D260000052600002B2600004F
:10253000292400002924000051250000292400003E
:10254000052600002924000029240000052600009B
:10255000BAF1000F0E9F35DB5146384606F01EFBE0
:1025600007EB000A002F3FF45FAF00269DF84230D2
:1025700013F01002059200F0938002305B06119A6E
:1025800048BF129B0492104448BFC018B8F1000F16
:1025900040F3A0809DF84020A8EB0008C2F3800320
:1025A0005007069300F19680510640F189803EB1B4
:1025B00059463046C84700287FDB069B01351E463A
:1025C00030227EE0384606F0E2FAC9E70E9B8DF82D
:1025D0002030002608AF0DF1210A0120C6E71907B7
:1025E0005CBFC3F300135E01DDE90E2348BF2B2659
:1025F000002BBFF662AF524263EB4303CDE90E23DB
:102600002D265AE7002658E700269DF840200DF1B8
:102610003603DB1B6FF386129A458DF840207FF658
:102620005AAFAAEB0303119355E70E9890B30DF13F
:102630003603009310AA08AB002106F017FABDF884
:10264000423003F0EF0343F4F04343F01003BAF1D8
:10265000000F0746ADF84230D6DA00283FF4E4AE6A
:102660000DF13603181A00269A467FE70E9B0729BC
:102670003FF6DAAEDFE801F00C04060C08080C0C9B
:102680001D70D1E61D80CFE6EA17C3E90052CBE604
:102690001D60C9E62E4F064607F1050A052065E7CD
:1026A0001A0748BF013069E707931046069259465A
:1026B000C8470028DDE9062304DA15B0BDE8F08F2D
:1026C000202243461946002903F1FF33ECDC454440
:1026D0006D1A98462EB159463046C8470028ECDBA3
:1026E00001359DF84230DA0601D41B0705D559465D
:1026F0003020C8470028E0DB0135059B33B19DF849
:1027000043005946C8470028D7DB0135049E2E44B4
:1027100005E059463020C8470028CEDB0135731B41
:10272000002BF6DC53463A465946484606F0E4F993
:102730000028C2DB0544A844A8EB0503002B7FF763
:1027400073AE59462020C8470028B6DB0135F3E7B1
:10275000DD9F000008B54FF02002EFF3118382F3F4
:102760001288BFF36F8F00F085FE034806F012F960
:1027700000F04CFAFCE700BFE39F00002DE9F843AE
:1027800005464FF02003EFF3118683F31288BFF361
:102790006F8F1C4804F09CFA40B91B491B488E22DD
:1027A00006F0C8F918488E2106F0BDF91548184FF3
:1027B000DFF8608004F0AAFA174B1C684FF00C0990
:1027C00094B9104804F092FA40B90F490F48B92261
:1027D00006F0B0F90C48B92106F0A5F986F3118886
:1027E000BFF36F8FBDE8F883D4E90123002D18BF34
:1027F00013462BB198F8142009FB02F2B85C9847F5
:102800002468DDE768080020B09F00002F9C0000CE
:10281000700800208C0F00207C0800200A4ABFF3BB
:102820005B8F430902EB830200F01F00012383400A
:10283000DB4352E8000F184042E800010029F8D1BC
:10284000BFF35B8F704700BF6C08002070B5194B59
:102850001C7DBFF35B8F04F01F0301229A40164BCF
:10286000610903EB8103D04353E8001F01EA00052F
:1028700043E80056002EF7D1BFF35B8F0A4213D016
:102880000E4B0F4D8BB10C236343EA18E85C517873
:1028900006F0C9F90020FFF771FF0C235C432A19E9
:1028A00000232B51C2E9013370BD83F31188BFF3BC
:1028B0006F8FEFE78C0F002084080020278C00002A
:1028C000700800202DE9F843324B334A1C7DBFF3DA
:1028D0005B8F63094FEA830852F823302F4EBFF312
:1028E0005B8F04F01F0943FA09F313F0010F074649
:1028F0000AD10146204600F069F828B107C80C2328
:1029000003FB046383E807000C236343F218F55CC0
:102910002DB92046FFF782FF2846BDE8F8837B1CCF
:1029200010D0D2F808C01E4D1E4A4FF400400021BE
:10293000ECFB005100232846FDF7E2FB0121381A89
:1029400005F0E2FC04F0B0FD0120FFF717FFBFF334
:102950005B8F154B9844012303FA09F358E8002FC5
:102960001A4348E800210029F8D1BFF35B8F0F4BD1
:1029700033B10C236343F218F05C517806F047F949
:10298000FFF764FF2046FFF749FF04F0E1FD012057
:10299000C3E700BF8C0F00206C08002070080020E7
:1029A0003F420F0040420F00840800200F8C0000BF
:1029B000054BBFF35B8F53F82000BFF35B8F0038EC
:1029C00018BF0120704700BF880800202DE9F74F8D
:1029D000884601A900F042F8441E24B204EB4404E6
:1029E000DFF86C900546A40025B92F46384603B0A1
:1029F000BDE8F08F019B185D1F19FFF7D9FF064650
:102A000010BB7868134A4FF4004ACC463146E0FBCD
:102A10000AC100236046FDF773FB8346B8680D4A80
:102A2000CC463146E0FB0AC100236046FDF768FB57
:102A3000094B1B685A1C01D0834205D9B8F1FF3FEE
:102A4000D4D058444045D1D9013DADB20C3CCBE780
:102A50003F420F0040420F00C404002008B9024B5F
:102A60000B600020704700BF68990000014805F026
:102A7000AFBD00BF6899000010B5044618B90D4BF2
:102A80000D485B689847616831F004030CD0082951
:102A90000AD011F0020108D00848214603F0F2FFE5
:102AA000002323600023636010BD2068142206F019
:102AB000A5F8F7E7640600200CA00000A40D002094
:102AC00008B508B34368042B10D101220368BFF393
:102AD0005B8F53E8001F002903D143E80020002842
:102AE000F7D1BFF35B8F0BD1002008BD53B1006855
:102AF0004FF0FF324FF0FF3304F03EF90028F3D0DF
:102B00000348F2E70348F0E76FF4E040EDE700BF69
:102B1000E98FFFFFEA8FFFFF08B5C0B14368042BC0
:102B200010D100220368BFF35B8F53E8001F012917
:102B300003D143E800200028F7D1BFF35B8F09D110
:102B4000002008BD43B1006804F0E8F9F8E76FF42D
:102B5000E040F6E70148F4E70148F2E7E98FFFFFBC
:102B6000EA8FFFFF10B5044618B9164B16485B688C
:102B700098476368042B23D0082B21D0CBB9236856
:102B8000BBB912484FF0FF324FF0FF33214603F03C
:102B90001FFF08B923681BB90A4B0D485B689847AB
:102BA00020681422002106F029F8636843F002032C
:102BB0006360206806F011FD636843F00103636001
:102BC00010BD00BF640600200CA00000A40D002072
:102BD00032A0000008B5064906484023142206F03A
:102BE000CBFCBDE808400449044805F051BD00BFD6
:102BF000A4080020A40D0020709900008499000012
:102C0000014910220A60704710ED00E072B64040A2
:102C100080F31188BFF36F8FBFF34F8F30BF62B661
:102C2000BFF36F8F704700BF72B6494081F31188C0
:102C300020BF80F3118862B6704700BF40B2002801
:102C400007DB044A4109012300F01F00834042F8DA
:102C50002130704700E100E040B200280CDB43095E
:102C6000064900F01F0020330122824041F8232052
:102C7000BFF34F8FBFF36F8F704700BF00E100E0DD
:102C8000054B420900F01F0053F82220012303FAEC
:102C900000F01040704700BF00E100E038B54D1C67
:102CA000072D044608D90E490E48572205F042FF69
:102CB0000B48572105F037FF60B20028ACBF00F188
:102CC0006040094B4FEA4515B8BF00F00F00EDB268
:102CD000AABF00F561401D5480F8005338BD00BF05
:102CE0005FA000002F9C000014ED00E030BFFFF754
:102CF000FDBF00BF0B4A08B50B4B22F07F029A6064
:102D0000BFF34F8FBFF36F8FD3F8882022F4700288
:102D1000C3F8882003F07CFD05F06EF900F0F8F9A7
:102D200003F0BAFD0000000000ED00E0094A0A4986
:102D3000936809689967094958674B6843F080535D
:102D40004B60002383F31188BFF36F8F9368986FF4
:102D5000704700BF8C0F0020649B000000ED00E076
:102D600012498A684FF030001044EFF3098C80E874
:102D7000F01F202080F31288BFF36F8F0C4F4FF0AD
:102D80000066CA698A603E60506F0023536780F313
:102D9000118804B5104600F057FABDE8044002F16E
:102DA000300090E8F01F8CF3098870478C0F0020EA
:102DB00004ED00E01EF0040F0CBFEFF30880EFF30A
:102DC0000980816911F8021C0229FFD001B505F0C4
:102DD000C5FE01BD42F8203C009B42F81C3C0A495C
:102DE000019B42F8183C029B42F8143C21F001017F
:102DF0004FF0807342F8043C42F8081C0023203A4C
:102E000002654367704700BF598A0000094A0346BC
:102E1000906870B113F1160F406E05D0A0F120023A
:102E20009A4205D8834203D2814228BF00207047CE
:102E3000002070478C0F002008B5094B98600D46A4
:102E4000144600F001FA204685F30988002163B694
:102E500081F31188BFF36F8F0022002305F0FCFD82
:102E60008C0F002001B572B60B4A906900281EBF76
:102E70000021916106F0A2FB62B6EFF30580A0F19C
:102E800010004FEAC0000549014409C99847BDE850
:102E900001400349084700008C0F002050970000B4
:102EA000A52E0000044B9968D869884203D00349D5
:102EB0004FF080520A6070478C0F002004ED00E054
:102EC0000D4B9A6A9A6A9A6A920508D59A6B9A6A21
:102ED000120404D518B19A6A22F400429A629A6ADE
:102EE0009A6AD205044A58BF9B6A936A002043F449
:102EF0007F4393620870704700ED00E0234B70B58C
:102F000014469A6A9A6A9A6A920705462AD5586BB5
:102F10009A6A160626D519B19A6A22F080029A6238
:102F20009A6A9A6A9A6AD10602D49B6A9A072AD543
:102F3000164E73681B0526D52946FFF767FFA0B11B
:102F400080F309880220114B9A6A920642BF5A6A9E
:102F500022F400525A629A6A42F0FF029A620023F7
:102F6000237070BD6FF01500DAE7B36AD9060AD591
:102F70000749084840F2491205F0DCFD044840F2D8
:102F8000491105F0D0FD0020DDE700BF00ED00E0B5
:102F900095A000002F9C000070B5514B5C688AB072
:102FA0000546C4F30804002686F31188BFF36F8F2B
:102FB00002F07F43B3F17F4F08D102F00C03082BDE
:102FC00004D010074CBF0D4601265DB9454946485F
:102FD00040F2FB3205F0AEFD424840F2FB3105F015
:102FE000A2FD002500238DF80730E31E032B45D8F2
:102FF000DFE803F002666A6E394BDA6A91073DD466
:10300000DA6A002A3ADBDA6A520050D5AA6932F845
:10301000021C4DF60272914201D12C682FE093F808
:10302000282032B10DF1070201212846FFF766FF83
:1030300007E093F8292032B10DF107010120FFF7D5
:103040003FFF04461BE05A8D92B262B19A6A9A6AB7
:103050009A6A9A6A9A6A9A6A9A6A6FEA02426FEA66
:1030600012429A620AE01F491F4840F2CD2205F041
:1030700061FD40F2CD211B4805F055FD00249DF86F
:10308000073093B92022294602A805F0ACFD099B20
:1030900006B3C3F3080222B96FEA53236FEA43234E
:1030A000099302A9204605F057FD0AB070BD0D49ED
:1030B0000D4840F2D12205F03DFD40F2D121DAE782
:1030C0000DF107020021B0E70DF107010020B6E77E
:1030D000034BBBE723F4FF7323F00103E0E700BFDA
:1030E00000ED00E095A000002F9C0000024A53690B
:1030F00043F010035361704700ED00E0EFF30880E8
:10310000EFF3098101B57246FFF746FF01BD00BF2D
:10311000044800232021C2180133302B82F8001309
:10312000F9D1704700E100E0002080F31488BFF37C
:103130006F8F06F07BFA00200D490860BFF34F8FB8
:103140000C4880F3088800F02BF8202080F31188C9
:1031500009484FF40261401880F30988EFF31480A6
:103160000221084380F31488BFF36F8FFFF7C2FD7D
:1031700094ED00E040230020C01500200749D1F85D
:1031800090200023C2F307221846934200DB7047C9
:10319000C1F89830C1F8A0000133F6E700ED00E077
:1031A00008B572B6002383F31388FFF7E7FF144BCB
:1031B0004FF0FF32C3F88020C3F88420C3F8882082
:1031C000C3F88C20C3F89020C3F89420C3F898204B
:1031D000C3F89C20C3F88021C3F88421C3F8882158
:1031E000C3F88C21C3F89021C3F89421C3F8982127
:1031F000C3F89C2162B6BFF34F8FBFF36F8F08BD3A
:1032000000E100E0084B9B6883420BD1EFF305839C
:1032100043B1064B5A6842F080525A605A6A22F40F
:1032200000425A6204F054BE8C0F002000ED00E012
:10323000024B034A0348012100F070B8000004204B
:103240000000002094990000426E054B203A1A605D
:10325000044A2021C3E901121846012100F07CB87C
:10326000C40D002000000B15F0B5204E00258D4246
:1032700001DB1046F0BD446874B353B104F1FF3C68
:1032800014EA0C0F2FD11F2C2DD907681CEA070F49
:1032900029D1202C0768D0F808C05FFA82FE1ED919
:1032A000B4F1004F1DD8013CB4FA84F4C4F11F04FA
:1032B0006400BEF1070F4CEA040C14D827F01F0479
:1032C000144344F01004C6F89820C6F89C404CF013
:1032D0000104C6F8A040013201350C30C7E70824CC
:1032E000E7E73E24E5E76FF01502C2E700ED00E0F6
:1032F000044B0522C3F89420BFF34F8FBFF36F8FA9
:10330000704700BF00ED00E0BFF35F8F024B00226B
:10331000C3F89420704700BF00ED00E010B50B4CDF
:1033200001232278FFF7A0FF207016300CD1084946
:10333000084840F2111205F0FDFBBDE810400448BA
:1033400040F2111105F0EFBB10BD00BFAC11002021
:10335000CFA000002F9C000008B50F4A0023127870
:10336000FFF782FF10F1160F03D00C4A07280DDD7E
:1033700008BD0B490B484FF4987205F0DBFBBDE824
:10338000084007484FF4987105F0CDBBC2F898008B
:10339000C2F8A0300130E9E7AC11002000ED00E0F8
:1033A000CFA000002F9C0000234910B50C68082C0A
:1033B0000DD9224922484FF4A47205F0BBFB1F48E7
:1033C0004FF4A47105F0AFFB4FF0FF3010BDFFF7D5
:1033D0009BFF48681B490022944200F10C000BD16E
:1033E000194B1C70FFF784FFD1F89030C3F307230B
:1033F000082B14D10020E9E7C1F8982050F80C3CC4
:1034000023F01F03134343F01003C1F89C3050F81E
:10341000043C43F00103C1F8A0300132DCE7074966
:1034200007484FF4D47205F085FB04484FF4D4717B
:1034300005F079FBDEE700BFA0990000CFA00000F7
:103440002F9C000000ED00E0AC1100204FF02002A6
:10345000EFF3118382F31288BFF36F8F044A0121C7
:10346000C2F8401583F31188BFF36F8F00207047B7
:1034700000E001404FF08043C0B2C3F81C05BFF329
:103480004F8F0549054BCA6802F4E0621343CB60D5
:10349000BFF34F8F00BFFDE700ED00E00400FA0529
:1034A00020B1034B800143F001031847704700BF70
:1034B0000099000037B50C460A490B4A411A4023CF
:1034C0000093491105462346084805F0C5FB011E37
:1034D00005DA2846234603B0BDE83040184703B05C
:1034E00030BD00BFE40D0020C58C0000A896000090
:1034F00038B5CCB2012C054608D9084908487922CC
:1035000005F018FB0548792105F00DFB2B690C220D
:1035100004FB0233986C00F0070038BD15A10000D1
:103520002F9C0000F8B5CCB2012C06690546174661
:103530000AD91949194840F24D1205F0FBFA16480C
:1035400040F24D1105F0EFFA4FF02003EFF3118236
:1035500083F31288BFF36F8F0C2101FB04639B6C14
:1035600013F0C00308D09F4206D082F31188BFF346
:103570006F8F4FF0FF30F8BD01FB04660123B36489
:1035800082F31188BFF36F8F6B6803EBC4035B6832
:1035900098470020EFE700BF15A100002F9C000016
:1035A00070B50D460649411A0446491105484022A6
:1035B000FFF7B8FF2B4601462046BDE8704018478C
:1035C000E40D0020A8960000002270B501210446F9
:1035D0001046FFF763FB0F4801F054FD0E4B984275
:1035E00015D101F071FD26690C49304605F021FA2C
:1035F00000280BDB246909490125B56404F120008A
:1036000005F017FA002801DB6565002070BD6FF03A
:103610000400FBE7553600000000AD0BC099000028
:1036200001460C2309484B4370B5C418D4E9105621
:10363000002248332264184405F0FBFA2DB13246CB
:103640002B460348BDE87040184770BDE40D0020CC
:10365000A8960000012808B506D0032808D0A0B914
:103660000F4B9B6C5B0719D1BDE80840FFF7D8BF33
:103670000C490D4840F25E2205F05CFA40F25E21F2
:10368000BDE80840074805F04EBA0649064840F232
:10369000622205F04FFA40F26221F1E708BD00BF57
:1036A000E40D002015A100002F9C000008B54FF08C
:1036B0002003EFF3118183F31288BFF36F8F124A57
:1036C000136843F002001060DA0708D481F3118810
:1036D000BFF36F8F0120BDE8084001F017BD4FF028
:1036E0008043D3F80C24D3F80C34D307EED5074825
:1036F00005F09FFA81F31188BFF36F8F0020BDE8BA
:103700000840FFF78DBF00BF3C0E00202C0E0020AC
:103710001FB500220123CDE90223094ACDF800D0CC
:103720006B46CDF804D005F0C6FA002805DB4FF44F
:1037300080420023684603F0BFFC05B05DF804FB3F
:10374000E38C0000094BBFF35B8F53E8002F22F09E
:10375000020143E800100028F7D1BFF35B8FD307C5
:1037600002D4012001F030BD704700BF3C0E0020A4
:10377000024BC0B203EB4010704700BFE40D0020C5
:103780002DE9F0414649BFF35B8F0646012251E81F
:10379000003F41E800200028F9D1BFF35B8F9BB9BF
:1037A000404941484B60CB608A60FEF79BFB002894
:1037B0000ADA3E493E484FF4087205F0BBF93B482F
:1037C0004FF4087105F0AFF976B3731E012B59D889
:1037D000012E07D14FF08043D3F81C3403F00303CC
:1037E000012B21D005F0E4FE0546F8B9314B1B78DA
:1037F000E3B14FF080430222C3F808230746DFF805
:10380000B8804FF08044D4F81834D4F81824D20388
:1038100016D503F00303012B01D0012E10D15DB3A7
:1038200087F31188BFF36F8FBDE8F0814FF020035D
:10383000EFF3118783F31288BFF36F8F0125DEE763
:10384000ADB13846FFF7F0F9D4F81835002BDAD1CE
:10385000D4F80421002AD6D0C4F80431D4F80431B5
:103860000123C4F81835C8F88031A360CBE70021E4
:10387000212004F0F7FAE7E74FF080430222C3F873
:103880000423D1E709490A4840F2322205F052F9EF
:10389000BDE8F041054840F2322105F044B900BFCF
:1038A000E00D0020D00D0020040E002015A1000026
:1038B0002F9C0000BD15002000E100E070B50569F7
:1038C00016460C4641B91E491E48242205F032F91D
:1038D0001B48242105F027F9636843B918491948A2
:1038E000252205F027F91648252105F01CF96B68FB
:1038F0004BB1A34213D1AA6823686B60944200D1F4
:10390000AB60002323607EB9002070BD9C4206D1CD
:1039100023681360AB689C42F3D1AA60F1E71A46B2
:103920001B68002BF2D13EB16B682360AB686C6002
:10393000002BE9D1AC60E7E76FF01500E5E700BFC9
:1039400058A100002F9C000030B54068057B01F0B5
:103950001F04B2F5001F85B044EA451404D1204687
:1039600001F03CFF002074E00025B2F5800FCDE9A6
:10397000025514D1B3F1007F0CBF042305238DF849
:1039800008300023194602AA204601F035FD3B4BC2
:10399000984270D10121204601F0B6FEE2E7B3F172
:1039A000C06F2CD0B3F1007F14BF012302238DF828
:1039B00008308368CB40D807E3D4B2F1A07FE0D1D0
:1039C000630904F01F0546D0012B1AD040F22922CA
:1039D0002B492C4805F0AEF8294840F2292105F082
:1039E000A2F82749274840F22E2205F0A3F840F21A
:1039F0002E21234805F097F84FF0A04312E003234F
:103A0000D5E74FF6FF73EB40D9070AD41C491D4890
:103A100040F2292205F08EF8194840F2292105F0DC
:103A200082F8194B05F5E07553F82530DB07A8D46B
:103A30000DF107052946204601F000FE134B984280
:103A400017D1284601F05AFE0C4B984211D06FF066
:103A50000B0005B030BD4FF0FF33EB40DA07CBD49D
:103A60000749084840F2292205F064F840F229216C
:103A7000BFE7039585E76FF00400EAE70000AD0BB0
:103A800085A100002F9C0000000300500400AD0B36
:103A900010B501F023FE044668B901F0F7FD084BAC
:103AA00098420AD10748214601F0C2FD224605216D
:103AB0000620FFF7F3F8002010BD6FF00400FBE7CD
:103AC0000000AD0BC93A00002DE9F843430903D0CB
:103AD000012B2AD0BDE8F883164F3B695C68002CA7
:103AE000F8D000F01F0001262568DFF84C80DFF8D1
:103AF0004C908640002CEDD0A3681E4210D0636825
:103B000043B941464846452205F014F84521404650
:103B100005F009F8D4E90132214632403846984789
:103B20002DB12B682C461D46E4E7054FD5E72B4603
:103B3000F8E700BFD896000058A100002F9C0000B5
:103B4000C09600002DE9F04347683B7B01F01F055C
:103B500085B00E4645EA43151446D2B902A9284657
:103B600001F06CFD0446284601F062FE464B984287
:103B700004D06FF0040005B0BDE8F083844201D0AA
:103B80000020F8E79DF8080001F0B2FDA042F7D050
:103B9000EFE74FF000090DF103013046CDE902993E
:103BA00001F04CFD4B46804602AA4946284601F0EA
:103BB00023FC354B984202D06FF01500DBE78045BF
:103BC00003D19DF8030001F093FDA3034CD540F20F
:103BD0000663234040F20622934219D00CD8062BEC
:103BE00017D004D8ABB1022BE6D1042311E0B3F512
:103BF000007FE1D101230CE040F20242934227D042
:103C0000B3F5C06F26D0B3F5806FD5D1022300E0A5
:103C100007238DF8043084F48033C3F30043E006B7
:103C20008DF8053054BFC4F34013032321038DF8EE
:103C3000063011D57A680123B340C2F80835002256
:103C400001A9284601F080FC0F4B984298D0B3E7B9
:103C50000523DEE70323DCE7620341BF01237A6823
:103C6000B340C2F80C35EAE7E3064FF0000354BF57
:103C7000C4F3401403241A4601A928468DF80440D1
:103C800001F0BAFBE0E700BF0000AD0B2DE9F04109
:103C900004680379276901259D4063681B681D42FC
:103CA0000E460AD11449154840F2924204F042FFF0
:103CB000114840F2924104F036FF3B681D426368B0
:103CC0001B6818BF86F001061D420AD10A490B483D
:103CD0004FF48D6204F02EFF07484FF48D6104F01D
:103CE00022FF36B1A368DB6829462046BDE8F041D3
:103CF0001847A3681B69F7E7FE9B00002F9C000094
:103D00002DE9F04F044687B0076900220121032006
:103D1000FEF7C4FF6368DC6905AA0021204605F0B0
:103D20000CFA00287BDB059B22681979186805F0DE
:103D30003CFA002873DBBC683C4EDFF8F490083492
:103D4000D7E9023203EBC203A4F10802934204D87C
:103D5000384605F023F8002061E054F8080C05F01F
:103D6000FDFB00285ED054F8088C14F804AC34F83D
:103D7000025CD8F808300193D8F80430029305F0BB
:103D80003003302BD8F810B00AD1314648464FF4F2
:103D90002E7204F0CFFE4FF42E71304604F0C3FEB5
:103DA00005F00603042B0AD1314648464FF4307221
:103DB00004F0C0FE4FF43071304604F0B4FEE80762
:103DC00054BF45F4B01585F4D015029A25F480133C
:103DD00012680393012303FA0AF313420CD14FF440
:103DE000357231464846029304F0A4FE4FF4357113
:103DF000304604F098FE029BDBF80020E9074CBF38
:103E0000134322EA0303CBF80030019B039A1B689B
:103E1000514640469847002804F1080490DA07B05C
:103E2000BDE8F08F6FF01200F9E700BFFE9B0000C5
:103E30002F9C0000034630B51D694068AA6C2B6DAD
:103E400085B02ABB8BB3696CAB6514461A46CDE9C5
:103E50000014E96C029131B3002B18BF1346002205
:103E60006946039301F034FF114B98420ED06FF076
:103E7000040400221146284604F06EFF2C6305F16D
:103E8000200003F0E3F8002385F85C3005B030BD76
:103E9000696C13B19A4228BF1A460029AA6514BF5B
:103EA00014460024D3E70B46D9E71C46E1E700BFE0
:103EB0000000AD0B2DE9F04F99468B8804698046D0
:103EC000980489B00E46924600F1C7804FF0FF3249
:103ED0004FF0FF3304F1100003F0EEF86660D8F8FD
:103EE00010B0D8F8043000939BF85D3001931BB1FB
:103EF000DBF800309E425FD0B788390500F1DC80E6
:103F000017F0090F40F0D580C7F34513082B40F098
:103F1000D0803568744B9D4240F2CB80009B03F10A
:103F2000080EBEE80F000DF10C0CACE80F00DEF837
:103F30000030CCF800306D4B9D4240F297806C4BC6
:103F40009D4240F296806B4B9D4240F295806A4BB9
:103F50009D4240F29480694B9D4240F29380684BB1
:103F60009D422CBF4FF000454FF08045BA070595A4
:103F700007F0040340F18980002B14BF03230223C0
:103F80008DF81830019BC7F300178DF819702BB10D
:103F9000009801F051FE00238BF85D305B46594AD2
:103FA000009803A901F08AFD574B984271D1012373
:103FB0008BF85D30CBF80060012384F85C30BAF1F7
:103FC000000F7CD1C4F834A00023A36304F148029D
:103FD00004F1380104F1340004F0ADFE6064B9F17D
:103FE000000F75D1C4F83C900023236404F1500203
:103FF00004F1400104F13C0004F09DFE002632462D
:10400000E06401212046266304F0A6FE4046FFF747
:1040100011FF256DA36C27469D4238BF1D464FF406
:10402000FA535D4357F8203B4FF4004C1B68B5FB37
:10403000F3F53146C83540F2E7304FF47A72002389
:10404000E5FB0C01FCF75CF802460B46384603F032
:1040500033F8002844D1256B1DE0A369002B7FF4C1
:1040600035AF636899427FF431AF38E74FF00075A0
:104070007CE74FF0806579E74FF0006576E74FF019
:10408000805573E74FF0005570E7003B18BF0123E0
:1040900076E76FF0040523689B8813F4005304D17E
:1040A000636004F1100002F0D1FF284609B0BDE8BA
:1040B000F08F6FF01505EEE76FF08505EBE7DAF8A6
:1040C00000306363002B3FF47FAFDAF804307CE705
:1040D000D9F80030E363002B86D0D9F8043084E7A8
:1040E0006FF07305D7E700BF47E801008FD00300EA
:1040F0001FA107003F420F007F841E00FF083D0004
:1041000000127A00E18D00000000AD0B2DE9F041B6
:1041100004680379276901259D4063681B681D4277
:104120000E460AD11449154840F2924204F002FDAD
:10413000114840F2924104F0F6FC3B681D4263686E
:104140001B6818BF86F001061D420AD10A490B48B8
:104150004FF48D6204F0EEFC07484FF48D6104F0DB
:10416000E2FC36B1A368DB6829462046BDE8F04191
:104170001847A3681B69F7E7FE9B00002F9C00000F
:104180002DE9F04F044687B00769002201212F2056
:10419000FEF784FD63689C6A05AA0021204604F0AE
:1041A000CCFF00287BDB059B22681979186804F096
:1041B000FCFF002873DBBC683C4EDFF8F490083449
:1041C000D7E9023203EBC203A4F10802934204D8F8
:1041D000384604F07BFE002061E054F8080C05F03E
:1041E000BDF900285ED054F8088C14F804AC34F8FB
:1041F000025CD8F808300193D8F80430029305F037
:104200003003302BD8F810B00AD1314648464FF46D
:104210002E7204F08FFC4FF42E71304604F083FCB4
:1042200005F00603042B0AD1314648464FF430729C
:1042300004F080FC4FF43071304604F074FCE80761
:1042400054BF45F4B01585F4D015029A25F48013B7
:1042500012680393012303FA0AF313420CD14FF4BB
:10426000357231464846029304F064FC4FF43571D0
:10427000304604F058FC029BDBF80020E9074CBFF5
:10428000134322EA0303CBF80030019B039A1B6817
:10429000514640469847002804F1080490DA07B0D8
:1042A000BDE8F08F6FF01200F9E700BFFE9B000041
:1042B0002F9C0000F0B504694668A56C236D85B09D
:1042C0008DB9002B36D11D4600221146204604F040
:1042D000DBFD256304F1200002F0B8FE002384F822
:1042E0005C3005B0F0BD616C03BB31BBB3680091BD
:1042F0009D4228BF1D46636CA5651BB1A36C002BB6
:1043000018BF2B460193E36C02931BB1236D002B66
:1043100018BF2B46002269463046039301F07AFF0E
:104320000E4B9842DDD06FF00405CDE79D4228BFCB
:104330001D46DAE7616C1D46D8E701F06043B3F132
:10434000005FD3D0082D28BF082504F15E072A4658
:10435000384604F048FC3946C8E700BF0000AD0B02
:104360002DE9F04F98468B880469074698048BB076
:104370000D46914600F1D8804FF0FF324FF0FF33E9
:1043800004F1100002F098FE6560D7F804B0D7F889
:1043900010A0DBF80C3003939AF85D3001931BB149
:1043A000DAF800309D426DD0AE88310500F1F18021
:1043B00016F0090F40F0EA80C6F34513082B40F0D1
:1043C000E5802B680293029A7D4B9A4240F2DE8090
:1043D0000BF1100EBEE80F000DF1100CACE80F0051
:1043E000DDE90223934228BF13469EE80300754A85
:1043F00093428CE8030040F2A080734A934240F25B
:104400009F80724A934240F29E80714A934240F2EA
:104410009D80704A934240F29C806F4A9342C0F064
:104420009B806E4A9342C0F09A806D4A93422CBFA3
:104430004FF0A0534FF02063B207069306F0040339
:1044400040F19080002B14BF032302238DF81C3011
:10445000019BC6F300168DF81D602BB1584601F084
:1044600067FE00238AF85D3053465E4A04A9584629
:1044700001F04CFD5C4B984278D101238AF85D3005
:10448000CAF80050012384F85C30B9F1000F40F005
:104490008380C4F834900023A36304F1480204F13C
:1044A000380104F1340004F0DEFC6064B8F1000F60
:1044B0007BD1C4F83C800023236404F1500204F152
:1044C000400104F13C0004F0CEFC00263246E064DA
:1044D00001212046266304F0D7FC3846FFF7EAFEA8
:1044E000256DA36C27469D4238BF1D464FF4FA53F5
:1044F0005D4357F8203B4FF4004C1B68B5FBF3F5C8
:104500003146C83540F2E7304FF47A720023E5FBBC
:104510000C01FBF7F5FD02460B46384602F0CCFDD8
:1045200000284AD1256B23E0A369002B7FF424AF38
:10453000636899427FF420AF27E74FF000737BE771
:104540004FF0806378E74FF0006375E74FF08053DA
:1045500072E74FF000536FE74FF080436CE74FF086
:10456000004369E7003B18BF01236FE76FF00405C4
:1045700023689B8813F4005304D1636004F1100096
:1045800002F064FD28460BB0BDE8F08F6FF0150512
:10459000EEE76FF08505EBE7D9F800306363002B99
:1045A0003FF479AFD9F8043076E7D8F80030E36308
:1045B000002B80D0D8F804307EE76FF07305D7E782
:1045C00047E801008FD003001FA107003F420F0002
:1045D0007F841E00FF083D0000127A000024F400D2
:1045E0000048E801118F00000000AD0BF0B54B79D9
:1045F000012B26D0032B21D110268B79032B1DD123
:10460000CC790CB1012C19D10A7912B1022A15D139
:104610000E220B684568B3F5164F2D6865D02DD86E
:10462000B3F5165F64D016D8B3F5966F62D00AD88A
:10463000B3F5967F61D0B3F5167F61D06FF085003A
:1046400052E00026D9E7B3F5166F5CD0B3F5965F5C
:10465000F4D1374B3CE0B3F5E14F57D007D8B3F571
:10466000615F55D0B3F5964FE8D1324B30E047F655
:104670001227BB42E2D14FF4000329E0B3F5613FBA
:1046800048D013D8B3F5963F47D009D84DF6C02788
:10469000BB4244D0B3F5614FD0D14FF46B0317E068
:1046A000B3F5E13FCAD14FF0EB7311E0B3F5612FE1
:1046B00038D008D8204FBB4237D0B3F5E12FBDD159
:1046C0004FF0E86304E01D4FBB42B7D14FF0805379
:1046D0000069C5F82435031D03C934432243C5F8D6
:1046E0006C2583E803000020F0BD4FF41D03EFE7C5
:1046F000134BEDE74FF49E23EAE74FF4A033E7E7CF
:104700004FF41C33E4E74FF41D23E1E70D4BDFE7E3
:104710000D4BDDE74FF06C73DAE70C4BD8E74FF445
:104720006503D5E74FF07063D2E74FF08063CFE7C2
:1047300000B0130000A04E0090D0030040420F00D4
:104740000050270000C0750000F03A0000903A01C8
:10475000F8B5066905460F4604F02AFFB0B92C4BA0
:104760001B789BB16424686804F037FCF8B9012019
:1047700004F08EFD013CF6D10021212003F072FBF4
:10478000F0E784F31188BFF36F8FF5E74FF0200354
:10479000EFF3118483F31288BFF36F8F686804F01E
:1047A0001CFC88B984F31188BFF36F8FEEE74FF0DC
:1047B0002003EFF3118483F31288BFF36F8F6868CF
:1047C00004F00BFC0028DCD006F8107F69680B6849
:1047D0000122C3F84465C3F848250022C3F820210C
:1047E000D3F82001C3F85821D3F858214A68D206DB
:1047F00041BF0822C3F800254FF48002C3F8042308
:1048000001229A6084F31188BFF36F8FF8BD00BF57
:10481000BD15002070B5012383400E4ABFF35B8FA6
:10482000DC4352E8001F01EA040542E80056002E6E
:10483000F7D1BFF35B8F4FF4803282400648C0F857
:104840000823BFF35F8FBFF36F8F0B4214BF0120AC
:10485000002070BD5C0E0020001001401B49F8B51F
:10486000044622F07F450868C1E90023A5F500133E
:10487000101AB3F5400F0FD303F086FDA30003F128
:10488000804303F58833D3F8402595421DD14FF47A
:104890000002C3F8402512E00D4B1B681A0A1B06E4
:1048A0005E190C4B42F10007C3E9006703F06CFD91
:1048B000094A04F5A87352F823309D4205D1064AEF
:1048C0004FF48033A340C2F84433F8BD40070020C2
:1048D000600E0020480700200010014011B3BFF314
:1048E0005B8F0123104A834052E800CF4CEA030C4F
:1048F00042E800C10029F7D1BFF35B8F0B4A4FF4A8
:1049000080338340C2F80433094BBFF35B8F1B68CD
:10491000BFF35B8FC340DB0742BF064B4FF400324F
:10492000C3F80021704700BF5C0E0020001001405A
:10493000580E002000E100E00D4B1868010A000647
:10494000BFF35F8F0B4BD3F80435181841F100010A
:10495000B3F5801F0AD2084BD3E90023904271EBD4
:10496000030303D210F1807041F10001704700BFD2
:10497000600E002000100140480700202DE9F74F8D
:1049800014461D460746FFF745FF0090FFF7D4FF8A
:10499000A04271EB05037AD2464B201A65EB010168
:1049A000984271F1000180F08180434B03EB0713C3
:1049B000D3E902239D4208BF944253D04FEA870AAD
:1049C0000AF1804A07F150090AF5883A4FEA890945
:1049D0001FFA89F924F07F4809F180494FF48033A8
:1049E000DAF84005354A09F58839BB404646D2F821
:1049F00004B5A0EB0B0020F07F402BF07F41012895
:104A0000CAF8401505D10193132004F009FE2B4A82
:104A1000019B0BF1020CA6EB0C0020F07F40B0F5DF
:104A2000000F88BF66460020C9F80000D9F80000D2
:104A3000C2F8443326F07F40CAF84005D2F8040596
:104A4000834506D0301A023820F07F40B0F5000FC1
:104A50001BD8A6EB080626F07F46361945F1000361
:104A600034461D4614490C983B0101EB0712C8500F
:104A70000D9B5360C2E90245002438460099FFF7B8
:104A80002DFF204603B0BDE8F08F3046AFE701238D
:104A90000B4ABFF35B8FBB4052E8000F184342E85C
:104AA00000010029F8D1BFF35B8FDBE76FF015043D
:104AB000E3E700BF010000013007002000100140C3
:104AC000580E002073B5194B194D00244FF0FF30DC
:104AD0004FF0FF31C5F80845C3E902014FF48033B8
:104AE000C5F80433134B02264FF400320121C5F8F8
:104AF00004631120C3F880212246FEF7CFF811206D
:104B0000FEF79CF80C4A0123AB602B6013600B4B43
:104B10000B4A0093019400232046FFF72FFF3046F5
:104B2000FEF72EFE204602B070BD00BF3007002009
:104B30000010014000E100E05C0E00205D48000034
:104B4000FFFF7F002DE9F743334CD4F804339A0775
:104B50000BD5D4F8043143B1304A0023C4F80431F2
:104B6000D4F804311368013313604FF02003EFF3DE
:104B7000118283F31288BFF36F8FD4F80433DB0301
:104B800029D5BFF35B8F264B53E8001F21F00100AE
:104B900043E80005002DF7D1BFF35B8F11B9D4F8BE
:104BA0004031C3B10025C4F84051D4F8403182F3FC
:104BB0001188BFF36F8FFFF7BFFE4FF02003EFF3B5
:104BC000118283F31288BFF36F8F164BD3E902670C
:104BD000B042B94106D282F31188BFF36F8F03B0A0
:104BE000BDE8F0834FF0FF384FF0FF39D3E90010F4
:104BF000C3E902891D604FF48033C4F8483382F35F
:104C00001188BFF36F8F0029E9D0009032463B46F0
:104C100028468847E3E700BF00100140600E0020EF
:104C2000580E002030070020431C13B521D0012866
:104C300021DDB0F5000F20DA441EFFF77DFE104B9A
:104C4000D3E90013421AB2F5000F0E4828BF002422
:104C500001322244824228BF024652184FF000001F
:104C600009490190009143F10003FFF787FE02B06C
:104C700010BD0448E0E70024DFE7024CDDE700BF99
:104C800040070020FFFF7F005D48000008B5FFF7E8
:104C900053FE024B1B68C01A08BD00BF400700202E
:104CA00003685A0910B504461CD0012A06D14FF6F4
:104CB000FF7203F01F03DA40D3070AD413491448E4
:104CC00040F2292203F036FF104840F2292103F078
:104CD0002AFF236803F01F025B09226005D14FF011
:104CE000A04010BD4FF0FF32E3E7012B0BD0074986
:104CF000074840F22E2203F01DFF044840F22E2107
:104D000003F011FFEBE70348EBE700BF85A10000CC
:104D10002F9C0000000300504FF08053D3F8302147
:104D2000082A06D1D3F83431052B02D8024AD05CC8
:104D300070470020704700BFE0A10000024AD2F88F
:104D40000034002BFBD0704700E0014008B54FF065
:104D50008053D3F83021082A4ED14FF080420021F1
:104D6000C2F80C11C2F81011C2F8381502F5404211
:104D7000D3F80414C2F82015D3F80814C2F8241587
:104D8000D3F80C14C2F82815D3F81014C2F82C1557
:104D9000D3F81414C2F83015D3F81814C2F8341527
:104DA000D3F81C14C2F84015D3F82014C2F84415E7
:104DB000D3F82414C2F84815D3F82814C2F84C15B7
:104DC000D3F82C14C2F85015D3F83014C2F8541587
:104DD000D3F83414C2F86015D3F83814C2F8641547
:104DE000D3F83C14C2F86815D3F84014C2F86C1517
:104DF000D3F84434C2F87035FFF78EFF18B1384B42
:104E0000384AC3F88C26FFF787FF18B1364BFB22D0
:104E1000C3F81825FFF780FF70B14FF080414FF0C5
:104E20008053D1F8E42ED3F8583222F00F0203F069
:104E30000F031343C1F8E43EFFF76EFF20B12B4B85
:104E40004FF40072C3F840264FF08053D3F830314E
:104E5000082B1AD14FF08043D3F80024D20744BF67
:104E60006FF00102C3F800244FF08053D3F83431BF
:104E7000052B02D81E4AD35C3BB14FF01023D3F868
:104E800008224FF08043C3F858254FF01021D1F885
:104E90000C32DB071FD517480123C0F80435FFF794
:104EA0004DFFD1F80C3223F00103C1F80C32FFF7AB
:104EB00045FF0023C0F80435FFF740FFBFF34F8FD5
:104EC0000D490E4BCA6802F4E0621343CB60BFF396
:104ED0004F8F00BFFDE70A4B0A4A1A6008BD00BFAA
:104EE000005000404881030000F000400090024064
:104EF000DAA1000000E0014000ED00E00400FA0546
:104F0000D80500200090D00370B501250268BFF3DA
:104F10005B8FB2FA82F3C3F11F03DBB205FA03F42D
:104F200022EA040450E8006F964204D140E8004CA5
:104F3000BCF1000FF6D1BFF35B8FE7D101480B70D6
:104F400070BD00BF0000AD0B0368CB40DB0710B5A0
:104F500014D401238B400268BFF35B8F43EA020144
:104F600050E8004F944204D140E8001CBCF1000F0F
:104F7000F6D1BFF35B8FEED1014810BD0148FCE7CD
:104F80000000AD0B0400AD0BF7B5044668B1012875
:104F90002BD038493848D82203F0CCFD3548D821E9
:104FA00003B0BDE8F04003F0BEBD4FF080430222E5
:104FB000C3F80823C3F80401D3F804210122DA60FE
:104FC000074601238DF8073042F210754FF08046F6
:104FD000C4B1012C36D0294927484FF44F7203F051
:104FE000A9FD26484FF44F71DAE74FF080430022C5
:104FF000C3F80803C3F80021D3F8002158600DF16D
:105000000707DEE79FB1D6F8183403F003033B60CF
:10501000D6F81834D80313D59DF80700012803D11A
:1050200004F036F9013DD3D1012C09D114E0D6F8B2
:105030001834D90304D5012004F02AF9013DF6D132
:1050400003B0F0BD67B1D6F80C3403F001033B7038
:10505000D6F80C34DA03DFD4094B00225A71EFE79B
:10506000D6F80C34DB03F7D5012004F011F9013D2B
:10507000F6D1F1E7E6A100002F9C000023A200007A
:10508000640E002010B5044650B90A490A4840F29F
:10509000151203F04FFD074840F2151103F043FDD0
:1050A000064B1A7922B9012205481C609A8010BD6E
:1050B0000448FCE7E6A100002F9C0000640E0020DD
:1050C0000000AD0B0C00AD0B08B50D4B1B7953B9AF
:1050D0000C490D484FF4977203F02CFD09484FF42A
:1050E000977103F020FD0020FDF7CAFD08B9FDF718
:1050F000A5FD4FF080430022C3F8182508BD00BF6E
:10510000640E0020E6A100002F9C00002B4B1B79B1
:1051100010B5044653B92A492A484FF4B47203F033
:1051200009FD27484FF4B47103F0FDFC74B1012C64
:1051300039D0234923484FF4D37203F0FBFCBDE878
:1051400010401F484FF4D37103F0EDBC4FF0804284
:10515000D2F81834D2F81814C80312D503F0030398
:10516000012B1AD14FF08042C2F818350023C2F843
:105170000431D2F804310223C2F8043301239360CE
:105180000AE0D2F81434D9070BD5D2F81C349B07A7
:1051900004D40223C2F8043310BD13B10020FFF77A
:1051A000F3FE0023DEE74FF080430022C3F8002126
:1051B000D3F80021C3F804431C60EDE7640E00201F
:1051C000E6A100002F9C00000A4B1B7910B5044695
:1051D00053B90949094840F2AD1203F0ABFC064847
:1051E00040F2AD1103F09FFC2046BDE81040FFF7F0
:1051F000CBBE00BF640E0020E6A100002F9C000083
:105200004FF0804310B5D3F800216AB10022C3F8F3
:105210000021D3F800210122C3F80823114B58794B
:1052200010B95A711B6898474FF08043D3F8042196
:1052300072B10022C3F80421D3F80421D3F8182452
:10524000D3F81814920704D10122C3F818259A60E4
:1052500010BD0222C3F80823024BBDE810401B68B2
:1052600001201847640E0020034B083033F810006B
:10527000C0F34010704700BFDC050020044B08302D
:1052800033F8100010F01C0018BF0120704700BF59
:10529000DC050020034B083033F81000C0F3400059
:1052A000704700BFDC05002070B500F108030C4C0E
:1052B00034F81330DA0505460E4607D5C3F3432309
:1052C00004EBC30254F8333052689847A3682BB1FB
:1052D000E26831462846BDE87040184770BD00BFFF
:1052E000DC05002010B50446006803F0D3FF50B978
:1052F0001149124840F2292203F01CFC0E4840F2EA
:10530000292103F010FC236803F01F025B092260CF
:1053100002D14FF0A04010BD012B0BD00649074829
:1053200040F22E2203F006FC034840F22E2103F047
:10533000FAFBEEE70248EEE785A100002F9C000093
:1053400000030050194A083010B532F81030D90562
:105350001DD5C3F3432123F4F85322F8103002F192
:105360000E04002034F8023F13F4807F03D0C3F30F
:10537000432399420BD001303028F3D1002342F867
:1053800031300B48FFF7E0FD0A4B984200D110BDC9
:1053900009490A484FF4997203F0CCFBBDE810406C
:1053A00005484FF4997103F0BEBB00BFDC05002037
:1053B000500600200000AD0B57A200002F9C0000FB
:1053C00038B50246FFF750FF094C02F1080540B11D
:1053D00034F8153007495B0B03F5A273002041F840
:1053E00023001046FFF7AEFF002324F8153038BD28
:1053F000DC05002000600040F0B5044685B017468B
:105400001D46D9B103F057FF00BB0B46CDE90000A4
:105410008DF80E008DF80F000DF10F020DF10E0149
:10542000204603F053FF434A04F1080132F81130DB
:1054300023F0020343F0010322F8113047B3204662
:105440003E787A68FFF726FF10B1B2B13A4821E002
:10545000384F04F1080C37F81C1021F02001C90462
:10546000C90C27F81C1042B1032EEFD813789EB94F
:10547000324A03F5A27342F823602E4A04F1080170
:1054800032F8113023F01C0343EA860322F811306E
:105490003DBB2B4805B0F0BD9A0002F1804202F5F9
:1054A000C04241EA4331D2F8100520F00300C2F8AF
:1054B0001005D2F8100520F44F3020F44070C2F8E7
:1054C00010052002D2F810E500F47C5040EA0640B6
:1054D00040EA0E0041F0200127F81C10C2F8100528
:1054E000CBE7D5E900672046FFF72CFF002ED0D090
:1054F000104DD5E90023964201D19F4218D01148A2
:105500000DF10F01FFF700FD0D4B9842C2D19DF840
:105510000F2045F8326005EBC20308345F6035F8B0
:10552000143043EA422343F4807325F81430B0E783
:105530000022EEE7DC0500200400AD0B0060004017
:105540000000AD0B50060020F0B5044685B01546AE
:1055500021B3FFF79FFE20B92046FFF785FE002804
:105560005ED12046FFF78AFE10B14B78012B57D051
:1055700001238DF80F300023CDE900134A1C8B1C4A
:1055800020460DF10F0103F0A1FE264A04F10801A7
:1055900032F8113043F0030322F8113015B92248D4
:1055A00005B0F0BD2046FFF775FEC8B31D4E95F857
:1055B00000C004F10807614636F81700890020F0A2
:1055C000200001F18041C00401F5C041C00C26F863
:1055D00017000023C1F810356A78002ADFD0D1F80F
:1055E0001035AD7823F4991323F4F853C1F810352E
:1055F000D1F810E5230203F47C53120402F4403284
:1056000043EA0E0313432A0502F4801240EA4C30A9
:10561000134340F0200026F81700C1F81035BEE70C
:105620000248BDE7DC0500200000AD0B0400AD0B17
:10563000014BC3E902017047DC05002038B5044680
:105640000D4651B90C490D4840F2352203F072FA6B
:10565000094840F2352103F066FA2046FFF704FEC0
:1056600038B1074B0748083433F814305B0B2B7004
:1056700038BD0548FCE700BF57A200002F9C000082
:10568000DC0500200000AD0B0400AD0B38B50F4C5D
:1056900094F87850BDB96022294604F1100003F057
:1056A000ADFA0620FDF7CAFA094B0A48C3F87C5147
:1056B000D3F87C214FF00042C3F80423012384F87F
:1056C0007830636738BD0448FCE700BFDC05002084
:1056D000006000400000AD0B0500AD0B034B93F8DC
:1056E0007800003818BF0120704700BFDC0500209B
:1056F00001460148FFF728BC4C060020014601483E
:10570000FFF702BC4C060020F7B504460D46FFF734
:10571000B5FD50B92D492E4840F2DF3203F00AFAA8
:105720002A4840F2DF3103F0FEF92046FFF79CFDE6
:10573000284E04F10807F8B12046FFF7ABFDD8B9B1
:1057400036F81720520B930003F1804101F5C24156
:1057500003F1804303F5C04308600968D3F81015CE
:1057600041F00101C3F8101525B1012393401A4AF5
:10577000C2F8043303B0F0BD55B91449144840F2DF
:10578000EE3203F0D7F9114840F2EE3103F0CBF9D5
:1057900036F81730C3F38203042B12D0052B12D036
:1057A00001A80194FFF79EFD019BD0F81015D94088
:1057B00001F001010231204603B0BDE8F04003F0E2
:1057C000D2BD0321F7E70221F5E700BF57A2000091
:1057D0002F9C0000DC0500200060004008B5024658
:1057E000FFF742FDC8B11046FFF754FDA8B90832D3
:1057F0000D4B0E4933F8123001225B0B9A409B008F
:1058000003F1804303F5C043C1F80823D3F8102502
:1058100022F00302C3F8102508BDBDE808400021AE
:10582000104603F0A0BD00BFDC0500200060004072
:105830000E4B00F1080213B533F81230DB070446B3
:1058400011D5FFF7CBFF2046FFF7BAFD01A8019461
:10585000FFF748FD019B03F5E073022240F8232087
:10586000034802B010BD0348FBE700BFDC05002081
:105870000000AD0B0400AD0B2DE9F04F694B6A48F9
:105880006A49002687B0012234461D6835B1D0F838
:10589000045315421EBF1C601D68164304338B421F
:1058A0004FEA4202F1D1DFF88091D9F87C31002B28
:1058B00000F09B804FF0A043D3F820250492C3F85A
:1058C0002025D3F820280592C3F820284FF000089F
:1058D0000DF1100A4FEA481300934FF0010B4BE013
:1058E000009B534A94FAA4F4B4FA84F41C44E008EC
:1058F00004F1080304F0070132F813701AF80030BD
:1059000003940BFA01F123EA0103BA080AF8003004
:1059100003A80192FFF7E6FC039B019A03F5E073ED
:10592000C7F3820550F8233052072F46C3F30143D3
:105930002CD539462046DDB2FFF7B6FC03A8039408
:10594000FFF7D0FC039B03F5E07350F82330C3F35B
:1059500001439D4207D10021204603F004FD294662
:10596000204603F000FD03A80394FFF7BBFC039B54
:105970000BFA03F3C0F820355AF82840002CAFD1B9
:10598000B8F1000F1DD14FF00108A3E7022B0CD195
:105990000321204603F0E7FC05F00503012BE2D1CB
:1059A00039462046FFF780FCDDE7022120460193BF
:1059B00003F0D9FC032DF3D0019B032BD3D1022D8F
:1059C000EDE74FF0A042C9F87C41D9F87C31194984
:1059D000D2F820350493C2F82035D1F8202505925D
:1059E0001343C1F820257FF471AF012416B907B025
:1059F000BDE8F08F96FAA6F3B3FA83F304FA03F244
:105A00009B0003F1804303F5C04326EA0206D3F866
:105A10001005D3F81015C0F30520C1F30141FFF7BD
:105A200043FCE3E70061004000600040206100406B
:105A3000DC0500200003005001460148FFF764BA6E
:105A40005806002003685A0910B504461CD0012AE4
:105A500006D14FF6FF7203F01F03DA40D3070AD4D2
:105A60001349144840F2292203F064F8104840F228
:105A7000292103F058F8236803F01F025B09226014
:105A800005D14FF0A04010BD4FF0FF32E3E7012BEE
:105A90000BD00749074840F22E2203F04BF8044888
:105AA00040F22E2103F03FF8EBE70348EBE700BF9D
:105AB00085A100002F9C0000000300502DE9F34752
:105AC000074691469A460C4641B9564956487C22AB
:105AD00003F030F853487C2103F025F897F8048050
:105AE000524D282000FB08F029180B7F002B40F0B6
:105AF00097803E68E37B45F80090C1F804A081F8E8
:105B00002530E2788A776279CA77227B002B3FD1F1
:105B1000012A20787BD803F076FC2378019301A832
:105B2000FFF790FF019B03F5E073012240F823206B
:105B30006078FF280CD003F066FC6378019301A81D
:105B4000FFF780FF019B03F5E073032240F8232059
:105B5000A378FF2B0CD001A894F80E900193FFF7C7
:105B600071FF019B03F5E0734FEA890240F823209F
:105B7000E078FF280CD003F053FCE378019301A8F0
:105B8000FFF760FF019B03F5E073032240F8232039
:105B9000237C93B963782178FF2B18BF1A46A3782A
:105BA000C6F8081508BF4FF0FF32FF2B08BF4FF0B3
:105BB000FF33C6F80C25C6F81035A368C6F824359F
:105BC000637B227B003B18BF0123022A22D0032AD9
:105BD00023D0012A01D143F00203C6F85435012332
:105BE000C6F80035282303FB08F3EB5823B13868C7
:105BF00040F30730FDF722F8282303FB0855002364
:105C00006B770B4801232B7702B0BDE8F08703F0D8
:105C100007FC82E743F00403DFE743F00603DCE719
:105C20000448F1E795A200002F9C00006C0E0020B4
:105C30000000AD0B0500AD0B70B5224C0679282392
:105C400003FB064305461B7F43B91F491F48C1227A
:105C500002F070FF1C48C12102F065FF2823734346
:105C60002D68E35833B145F30730FCF7F5FF042303
:105C7000C5F808330023C5F80035282303FB064385
:105C800093F82530BBB9D5F8080503F0AEFBD5F87D
:105C90001005421C01D003F0A8FBD5F80C05431CED
:105CA00001D003F0A2FB282303FB0643987FFF28C3
:105CB00001D003F09AFB282303FB0644002323773B
:105CC00070BD00BF6C0E002095A200002F9C00004C
:105CD0002DE9F843504D0779282303FB07538146EC
:105CE0001B7F0C46904653B94C494D484FF4B37254
:105CF00002F020FF49484FF4B37102F014FF23680B
:105D000063B9636853B14549454840F2671202F0F0
:105D100011FF424840F2671102F005FFA36863B922
:105D2000E36853B13D493E484FF4B47202F002FFBC
:105D30003A484FF4B47102F0F6FE28237B43EA1888
:105D4000517F002966D1EB580BB10123537794E8BA
:105D50000F00282606FB075606F10C0C8CE80F00F6
:105D6000B07F0023FF2886F8243001D003F04BFBDE
:105D70002823B8F1000F06D003FB0753002229485F
:105D80005A77BDE8F883D9F8006003FB0753042273
:105D9000C6F80823C3F82080C6F80881D6F8082181
:105DA00062686AB12368012A1978C6F81C150BD1FC
:105DB000E368012B0BD9282303FB0753DB7F04E0A7
:105DC000DB7FC6F81C35F3E75B78C6F81C35282363
:105DD0007B43EC5824B10423C6F804331248D0E7BF
:105DE00007EB870105EBC101D6F80831002BFBD08A
:105DF000C6F808413046D6F8083103F0C3FA002847
:105E0000F2D1282303FB0755A87FFF28E6D003F033
:105E100007FBE3E70548B4E76C0E002095A20000FD
:105E20002F9C00000300AD0B0000AD0B0B00AD0B71
:105E300010B5134C236853B91249134840F29B1212
:105E400002F078FE0F4840F29B1102F06CFE0F4802
:105E50000B490023C0F80831D0F8083103F092FA5A
:105E600068B9A07FFF2801D003F0DAFA002323727B
:105E700063770748D4E90031BDE81040184710BDEA
:105E80006C0E002095A200002F9C00000030004006
:105E9000740E002003685A0910B504461CD0012A6C
:105EA00006D14FF6FF7203F01F03DA40D3070AD47E
:105EB0001349144840F2292202F03CFE104840F2F7
:105EC000292102F030FE236803F01F025B092260E3
:105ED00005D14FF0A04010BD4FF0FF32E3E7012B9A
:105EE0000BD00749074840F22E2202F023FE044857
:105EF00040F22E2102F017FEEBE70348EBE700BF6C
:105F000085A100002F9C0000000300502DE9F347FD
:105F10008046924699460C4651B97F497F484FF4D6
:105F2000BF7202F007FE7C484FF4BF7102F0FBFD28
:105F300098F804607A4F07EB46131B7F002B40F064
:105F4000E680002E40F0E580E07C2379627CD8F882
:105F50000050A16840EA430343EA8203BA7FC7E9DD
:105F600000A903F0070322F007021343BB77E3788D
:105F7000FB7700285DD1237B2078B1F1A05F08BFBB
:105F80000326012B00F2AD8003F057FA237801932A
:105F900001A8FFF77FFF019B360203F5E07346F08F
:105FA000010240F823206078FF280DD003F045FA65
:105FB0006378019301A8FFF76DFF019B03F5E07380
:105FC00046F0030240F82320A378FF2B0CD001A851
:105FD00094F80E900193FFF75DFF019B03F5E073CA
:105FE00046EA890240F82320E078FF2810D0237980
:105FF000002B79D003F021FAE378019301A8FFF791
:1060000049FF019B03F5E07346F0030240F82320AB
:10601000E07BFF280DD003F01DFAE37B019301A87C
:10602000FFF738FF019B03F5E07346F0030640F8E5
:106030002360237D53BB63782178FF2B18BF1A465A
:10604000A378C5F8081508BF4FF0FF32FF2B08BF33
:106050004FF0FF33C5F80C25C5F8103598F804301B
:10606000A3B9E378FF2B42D0627C002A3FD021798C
:10607000A27CC5F81435C5F86815C5F86425E37B1E
:10608000FF2B08BF4FF0FF33C5F86C35237CC5F8F4
:106090006035A368C5F82435637B227B003B18BFBD
:1060A0000123022A2DD0032A2ED0012A01D143F048
:1060B0000203C5F85435A379C5F8C0350723C5F8E0
:1060C00000353B682BB1D8F8000040F30730FCF7EF
:1060D000B5FD00237B77134801233B7702B0BDE871
:1060E000F08703F0B7F951E703F0B4F984E74FF014
:1060F000FF33C5F814350023C5F86835C5F8643595
:10610000BDE743F00403D4E743F00603D1E70648B4
:10611000E4E70648E2E700BFD0A200002F9C0000A1
:10612000940E00200000AD0B0500AD0B0300AD0B7D
:106130002DE9F341324D03795E0105EB4313074628
:106140001B7F53B92F49304840F20F2202F0F2FC76
:106150002C4840F20F2102F0E6FCAB593C6805EBFD
:106160000608CBB144F30730FCF776FD274BC4F8A3
:10617000083398F81D307BB1012363614FF0640848
:10618000D4F804312BB9012003F082F8B8F10108EA
:10619000F6D1AB1900225A770023C4F80035AB19A9
:1061A0009B7FDB071FD4D4F8080503F070F9D4F8FF
:1061B000100503F06CF9D4F80C0503F068F93B798D
:1061C0001BB9D4F86C0503F062F9AB19DB7FFF2B28
:1061D00009D001A80193FFF75DFE019B03F5E07371
:1061E000022240F823200A4B9C4208BF0123354479
:1061F00008BF636000232B7702B0BDE8F08100BFC9
:10620000940E0020D0A200002F9C00005201080034
:1062100000F002402DE9F047634F037907EB431983
:106220005E0199F81C3080460C46154653B95F490B
:106230005F4840F2DE2202F07DFC5C4840F2DE2145
:1062400002F071FC236863B9636853B15749584839
:1062500040F2DF2202F06EFC544840F2DF2102F0EF
:1062600062FCA36863B9E36853B1504950484FF4E6
:10627000387202F05FFC4D484FF4387102F053FC65
:1062800098F804303BB9E368B3F5803F03D2636804
:10629000B3F5803F0AD34549454840F2E12202F078
:1062A00049FC424840F2E12102F03DFC15F0080AA9
:1062B00011D0BB199A7F52070DD4DB7FFF2B0AD078
:1062C0003A493B484FF4397202F034FC37484FF4F6
:1062D000397102F028FCBB195A7F002A62D1BA59E1
:1062E00022B115F0140F04BF01225A7794E80F0071
:1062F00007EB060C0CF10C0C8CE80F000121484652
:1063000003F0B5F82168D8F8003021B101F06042FF
:10631000B2F1005F06D1A26852B102F06040B0F164
:10632000005F05D03E44002322487377BDE8F08724
:106330006068C3F84415C3F84805E168C3F834251C
:106340000022C3F83815C3F81821D3F8182115F026
:10635000010218BF0122C3F8502515F0020218BF30
:106360000122C3F84025BAF1000F07D0BA5972B91B
:106370000021484603F07BF80F48D7E701221A6155
:10638000BA5922B9D3F81821002AFBD0F0E715F04A
:10639000040F4FF0400202D0C3F80823ECE7C3F823
:1063A0000423E9E70548C1E7940E0020D0A20000CD
:1063B0002F9C00000A00AD0B0000AD0B0B00AD0BD5
:1063C000124BD3F8182110B5FAB1114C0022C3F8C2
:1063D0001821D3F81831236853B90E490E4840F2FA
:1063E0003B3202F0A7FB0B4840F23B3102F09BFB33
:1063F0000748002103F03BF8002323726377074826
:10640000D4E90031BDE81040184710BD00F002404B
:10641000940E0020D0A200002F9C00009C0E0020B3
:106420002DE9F0410546077990460C4641B93F49B0
:106430003F48532202F07EFB3C48532102F073FB9D
:10644000B8F1000F08D139493948542202F072FBE3
:106450003648542102F067FB364E0C2303FB0763DA
:106460001B7A002B60D12B68334A93420FD002F580
:10647000805293420BD002F58052934207D002F52E
:106480008032934203D002F58052934202D1A37826
:10649000032B08D925492648612202F04BFB2348EB
:1064A000612102F040FB0C237B43F21846F8038085
:1064B000636853606979286800239C46DAB2914288
:1064C0002AD840F30730FCF7B9FB2B686278D3F881
:1064D00004151A4821F0030102F003020A43C3F82D
:1064E0000425D3F80815A27821F0030102F0030275
:1064F0000A43C3F80825D3F81015227821F00F01BC
:1065000002F00F020A43C3F810250C2303FB0766B1
:1065100001233372BDE8F0819A0002F5A0720133C5
:1065200040F802C08258C9E70548F3E70CA3000011
:106530002F9C0000B40E0020008000400000AD0B36
:106540000500AD0B38B50E4D03790C2202FB035349
:1065500004461B7A012B08D00A490B488F2202F00F
:10656000E9FA08488F2102F0DEFA236801221A6056
:1065700023790C2202FB035502232B7238BD00BF86
:10658000B40E00200CA300002F9C000038B50D4D68
:1065900003790C2202FB035304461B7A43B90A49D0
:1065A0000A48972202F0C6FA0748972102F0BBFA80
:1065B00022680123136122790C2101FB02552B7201
:1065C00038BD00BFB40E00200CA300002F9C0000BB
:1065D00038B50D4C03790C2202FB034305461B7AA8
:1065E00043B90A490A489F2202F0A4FA07489F21AA
:1065F00002F099FA2B790C2202FB0344207A831EC5
:106600005842584138BD00BFB40E00200CA3000012
:106610002F9C000010B50A4B02790C2101FB0233BC
:1066200004461B7A43B907490748B32202F082FAAD
:106630000448B32102F077FA23680122DA6010BD22
:10664000B40E00200CA300002F9C00000249034858
:10665000042202F02CBF00BFB40E002000800040D6
:1066600002490348042202F022BF00BFC00E0020EE
:106670000090004002490348062202F018BF00BF04
:10668000D80E002000A0014010B5144C144A154942
:10669000032323616361144BA261E3614FF48063C0
:1066A00023620023A3626362E36222660F4A62668A
:1066B0001022A266E01D2367E366636702F05DFABD
:1066C000BFF35F8F0A49204602F057FABFF35F8F8E
:1066D0002023A371BFF35F8F10BD00BFE40E002025
:1066E00049A3000052A30000BD110020AD110020FD
:1066F00056A300000E4B70B553F82040013053F8FC
:106700002060A64200D870BDD4E9003528469847DD
:1067100065B1EB6830B10028B8BF4042FF28A8BF80
:10672000FF2018705A7842F001025A700834E8E7E6
:10673000509B000070B5054610B90024204670BD7E
:106740000378002BF9D00E4C0E4EB44208D10C4CFD
:10675000B442F2D0204602F001FF50B91834F7E7F6
:10676000204602F0FBFE10B12368AB42E6D018349D
:10677000EBE72168284602F01AFA0028EED1DDE79F
:10678000A896000050970000F8B504460E464FF05A
:106790002003EFF3118783F31288BFF36F8F01F0AB
:1067A00091FB31460546204602F062FD042C08D1DB
:1067B000084909488F2202F0BDF906488F2102F0EE
:1067C000B2F987F31188BFF36F8F2846BDE8F84010
:1067D000FCF718BD5DA300002F9C000008B50A4B14
:1067E000012202201A70FFF785FF02F01DFF03202F
:1067F000FFF780FF00F0F0F9FAF738FA034A137B4D
:1068000023F00103137308BDBD150020D00700203D
:1068100008B50348034A0021121A02F0A9FE08BD78
:1068200030070020C015002070B5002386B001227B
:10683000CDE90423134E144D01930F22CDE902320A
:106840001249182303FB005506EBC01604464FF40B
:10685000B07000FB04110E4B00954FF4A07230464F
:1068600000F062F9737B0B4AEE6023F0040373734C
:106870004FF4026304FB033313442C756B6006B0C2
:1068800070BD00BF500700208C0F0020E01D0020CD
:106890001D6D0000C015002080B52D4BA6B083F300
:1068A00008882C4D2C4E6B692C4F43F40073002448
:1068B0006B61E02385F82230EC772C766C76AC7631
:1068C00085F820406B6A43F4E0236B6285F823402F
:1068D000FCF70CFCFCF794F94FF0FF33AB62EB6272
:1068E000FCF762FDFCF7A4FC40F20113ADF8243084
:1068F00006ABB360CDE91F44229402F02EFE204681
:10690000FFF7F8FE0120164DFFF7F4FE01F096F9AF
:10691000144BF5610593012313490094CDE903431A
:106920004FF480623B46CDE90144284600F0FCF874
:106930006A7B064622F0040228466A7300F006FDD0
:106940002046FFF771FF3A4631462846FCF774FAB5
:10695000E01D002000ED00E08C0F0020DD6700004E
:10696000D00700207FA30000401F0020F8B5144C82
:10697000144D154EAC4208D9144831463D2202F060
:10698000D9F83D21304602F0CEF8AC4201D30020C8
:10699000F8BDD4E9041242EA010313F003030BD15A
:1069A000E068A361834201D12034E3E7A76917605F
:1069B0000133A2610A44F5E76FF01500E8E700BF74
:1069C000E0060020E006002084A300002F9C0000C9
:1069D0002DE9F74304460D4690461F4600F1080690
:1069E0004FF02003EFF3118983F31288BFF36F8F09
:1069F000304600F06DF940B91F4920488E2202F060
:106A000099F81D488E2102F08EF8304600F07EF98C
:106A1000A369C3B12B601B68A361E3690133E36120
:106A20000024304600F062F940B913491348B922F6
:106A300002F080F81048B92102F075F889F3118846
:106A4000BFF36F8F13E058EA070203D12B606FF09A
:106A50000B04E6E72246CDE900874946304600F0C0
:106A600049FF044618B9064B9B685B692B602046BA
:106A700003B0BDE8F08300BFB09F00002F9C000072
:106A80008C0F00202DE9F04104460D4600F1080668
:106A90004FF02003EFF3118783F31288BFF36F8F5A
:106AA000304600F015F940B91D491E488E2202F00B
:106AB00041F81B488E2102F036F8304600F026F9E6
:106AC000D4F81880B8F1000F0FD1204601F076F805
:106AD00058B12A684261C0F8788000F037FC394626
:106AE0003046BDE8F04100F067BC2B68A2691A602F
:106AF0002B68A361E369013BE361304600F0F6F8DF
:106B000040B907490748B92202F014F80448B921EE
:106B100002F009F887F31188BFF36F8FBDE8F081A9
:106B2000B09F00002F9C00002DE9F04385B0044683
:106B3000DDF83C80B8F10F0F0F461546994632D16B
:106B4000214B994533D104F15803C4E91633109B06
:106B5000237307350423637325F0070507F120032A
:106B6000C4E9193500260E9B84F80E80C4E9066638
:106B7000A660E673E66605F1200802930D9B01937B
:106B8000B8440C9B009342464B4639462046FCF7DE
:106B900021F90E4B66659B6803B11B6F2367404666
:106BA00005B0BDE8F08308F110031E2BCBD90849CE
:106BB000084840F2FF1201F0BDFF054840F2FF1106
:106BC00001F0B1FFBFE700BF1D6D00008C0F00207A
:106BD000A9A300002F9C00002DE9F043374C384D4D
:106BE000384F87B0AC4226460AD93748394640F27A
:106BF000D52201F09FFF40F2D521384601F093FFE6
:106C0000AE4204F130041BD300F04EFC2B4C2D4E51
:106C1000DFF8B480DFF8B490AC420AD93146404680
:106C20004FF43D7201F086FF4FF43D71304601F0A4
:106C30007AFFAC4220D307B0BDE8F04300F088BC37
:106C400054F8043C059354F8103C049354F8143C55
:106C5000039354F8183C029354F81C3C019354F8E5
:106C6000203C009354E90A2354E90C01FFF75CFF30
:106C700054F8303C5E65B5E7636A5A1C0FD023EACE
:106C8000E3734FF4004240F2E7300021C3FB0201FE
:106C900051EAC333276804D1384600F0C3FB3034CF
:106CA000BAE74FF47A720023F9F72AFA02460B4644
:106CB00007F11800494601F005FAF0E7E006002068
:106CC000E0060020A9A300002F9C00002D7B0000FF
:106CD000006838B1044B1B7D00F00300C01A18BFD8
:106CE00001207047012070478C0F0020064A117D5B
:106CF00092680A430168034691424FF0000004BFC6
:106D000018600120704700BF8C0F0020024B1A7DD5
:106D10009B681343036070478C0F0020124C08B52A
:106D2000A36893F90E30002B08DA10491048272287
:106D300001F000FF0D48272101F0F5FE0D4D4FF049
:106D40002002EFF3118382F31288BFF36F8F01F0FB
:106D5000A5FA2B78A06113B9FBF758FFEFE7FBF713
:106D6000B1FD0028EBD1F7E78C0F0020CCA3000089
:106D70002F9C0000BD1500202DE9F3410446174665
:106D80001E46EFF3058343B15F496048652201F079
:106D9000D1FE5D48652101F0C6FE4FF02003EFF300
:106DA000118883F31288BFF36F8F5948FFF790FF64
:106DB00040B9584955488E2201F0BCFE55488E21F5
:106DC00001F0B1FE5248FFF7A1FFE368524AE3B178
:106DD000A0689168884233D057EA060332D14C4804
:106DE000FFF784FF40B94B494848B92201F0A2FEA1
:106DF0004848B92101F097FE88F31188BFF36F8FDF
:106E00006FF00F0002B0BDE8F081916891F90E10AB
:106E10003F4821610133E3609368A360FFF766FF99
:106E200040B93C493948B92201F084FE3948B921BA
:106E300001F079FE88F31188BFF36F8F0020E1E73E
:106E40002169E5E791F90E1090F90E309942A8BF3B
:106E500019466FF07E029142B8BF11468B4249DD60
:106E600002F0B3FB0546CDE90076294822464146AB
:106E700000F040FD0028E1D04FF02003EFF3118631
:106E800083F31288BFF36F8F2148FFF721FF40B9CA
:106E900020491E488E2201F04DFE1E488E2101F031
:106EA00042FE1B48FFF732FF236821699C420AD04B
:106EB0004BB193F90E309942A8BF19466FF07E038B
:106EC0009942B8BF1946A06802F07FFBA0B99DB9EE
:106ED0000F48FFF70BFF40B90E490C48B92201F0EB
:106EE00029FE0C48B92101F01EFE86F31188BFF37C
:106EF0006F8F05E00025B6E70548314600F05CFAE3
:106F00006FF00A007EE700BFEDA300002F9C000099
:106F1000B40F0020B09F00008C0F002038B504464D
:106F2000EFF3058343B143494348C72201F002FE12
:106F30004048C72101F0F7FDA368002B74D03F4DF6
:106F4000AA68934273D1E36843B93A493A48DF22C9
:106F500001F0F0FD3748DF2101F0E5FDEFF3058397
:106F600043B137493448FD2201F0E4FD3448FD21A6
:106F700001F0D9FDAB68DB7B012B08D130492E48ED
:106F8000FE2201F0D7FD2E48FE2101F0CCFDAA68BB
:106F9000D37B013BD373E368012B05D9013BE3604D
:106FA00000F0D6FA002038BD4FF02003EFF3118532
:106FB00083F31288BFF36F8F2248FFF789FE40B931
:106FC00021491D488E2201F0B5FD1F488E2101F098
:106FD000AAFD1C48FFF79AFE2169A06802F0F5FAA5
:106FE000204600F0EBFDA06058B190F90E20226120
:106FF0000022826700F0AAF91248294600F0DCF965
:10700000CEE7E0600F48FFF771FE40B90E490A482D
:10701000B92201F08FFD0C48B92101F084FD85F300
:107020001188BFF36F8FBBE76FF01500BBE74FF020
:10703000FF30B8E7EDA300002F9C00008C0F00206C
:107040000FA40000B40F0020B09F000038B5044624
:107050004FF02003EFF3118583F31288BFF36F8F96
:107060001248FFF735FE40B9114912488E2201F04F
:1070700061FD0F488E2101F056FD0C48FFF746FEDA
:10708000204600F09BFD48B10022826700F05EF9C7
:1070900029460648BDE8384000F08EB9D4E90232EE
:1070A0009A4218BF0133A360F2E700BFB80F002077
:1070B000B09F00002F9C0000F7B5044617461D4600
:1070C000EFF305835BB152EA050308D02B492C4846
:1070D000792201F02FFD2948792101F024FD4FF09C
:1070E0002003EFF3118683F31288BFF36F8F2548D7
:1070F000FFF7EEFD40B9244921488E2201F01AFD28
:1071000021488E2101F00FFD1E48FFF7FFFDA36807
:10711000ABB1013B1B48A360FFF7E8FD40B91A493A
:107120001748B92201F006FD1748B92101F0FBFC10
:1071300086F31188BFF36F8F002003B0F0BD57EACC
:10714000050313D10F48FFF7D1FD40B90E490C4894
:10715000B92201F0EFFC0C48B92101F0E4FC86F300
:107160001188BFF36F8F6FF00F00E6E7CDE9007570
:1071700022463146034800F0BDFBDEE73AA400009A
:107180002F9C0000B80F0020B09F000038B5074DBD
:107190002C6854B1FDF77AFD054B04441C61286846
:1071A0000021BDE8384001F0AFB838BDC40F002061
:1071B0008C0F002038B5144D2B4653F8204F9C42BD
:1071C00000D004B9EC68AB6820B1AB68A34217D11A
:1071D000234613E043B90D490D48892201F0AAFC6A
:1071E0000A48892101F09FFCAB685A7BD206ECD19A
:1071F000A269002AE9D1DA897F2AE6D9EB6138BD94
:107200002046FFF7C3FFE3E78C0F00205AA40000DD
:107210002F9C000070B590F90D20437B002A044696
:1072200037DBDA0635D18569002D32D163F07F0373
:107230004373184B984208D117491848BA2201F0F5
:1072400079FC1548BA2101F06EFC154A134653F833
:10725000201F994218BF0D46516A25B9C4E9003173
:107260000C6054620CE094F90E0095F90E60B04287
:107270000BD0864209DD6B68C4E900531C606C606A
:10728000BDE870400020FFF795BF8D42E6D02D6825
:10729000E3E770BD500700205AA400002F9C0000B7
:1072A0008C0F0020F8B504460D464FF02003EFF395
:1072B000118783F31288BFF36F8F1E48FFF708FD15
:1072C00040B91D491D488E2201F034FC1A488E2118
:1072D00001F029FC17480026FFF718FD4FF4004C79
:1072E00040F2E73031464FF47A720023E4FB0C01A0
:1072F000F8F706FFB44202DD0228B8BF0220104AA8
:10730000104B1060104A98681E611560FFF73EFF31
:107310000848FFF7EBFC40B907490848B92201F0DB
:1073200009FC0548B92101F0FEFB87F31188BFF382
:107330006F8FF8BDC80F0020B09F00002F9C000089
:10734000C40F00208C0F0020C00F002038B5044669
:107350004FF02003EFF3118583F31288BFF36F8F93
:107360001248FFF7B5FC40B9114912488E2201F0CE
:10737000E1FB0F488E2101F0D6FB0C48FFF7C6FC5D
:107380002046FFF747FF0948FFF7B0FC40B908491E
:107390000848B92201F0CEFB0548B92101F0C3FB32
:1073A00085F31188BFF36F8F38BD00BFC80F002071
:1073B000B09F00002F9C000010B503460C46C1B9D9
:1073C000EFF30582AAB9144AD1699268914210D0AC
:1073D000FFF78CFC40B911491148D02201F0AAFBFB
:1073E0000E48D02101F09FFBBDE810400020FBF7C4
:1073F0009DBC1846FFF77AFC40B908490848B922F5
:1074000001F098FB0548B92101F08DFB84F3118848
:10741000BFF36F8F10BD00BF8C0F0020B09F000026
:107420002F9C000038B504464FF02003EFF3118580
:1074300083F31288BFF36F8F1848FFF749FC40B9F8
:10744000174918488E2201F075FB15488E2101F06E
:107450006AFB1248FFF75AFC637B5A0711D40F48A6
:10746000FFF744FC40B90E490E48B92201F062FB17
:107470000B48B92101F057FB85F31188BFF36F8FDB
:1074800038BD23F0040320466373FFF7C3FE29468B
:107490000248BDE83840FFF78FBF00BFC80F00208B
:1074A000B09F00002F9C000038B54FF02003EFF391
:1074B000118583F31288BFF36F8F2048FFF708FC14
:1074C00040B91F491F488E2201F034FB1C488E2111
:1074D00001F029FB1948FFF719FCEFF3058343B1CD
:1074E00019491848FD2201F025FB1748FD2101F03C
:1074F0001AFB164CA368DB7B012B08D112491148FB
:10750000FE2201F017FB1048FE2101F00CFBA268DF
:10751000D37B013BD3730948FFF7E8FB40B9084927
:107520000848B92201F006FB0548B92101F0FBFA31
:1075300085F31188BFF36F8F38BD00BFC80F0020DF
:10754000B09F00002F9C00000FA400008C0F0020B3
:1075500038B54FF02003EFF3118583F31288BFF3A2
:107560006F8F2448FFF7B4FB40B9234923488E228C
:1075700001F0E0FA20488E2101F0D5FA204C1D4898
:10758000FFF7C4FBA368DB7B53B91E491B4840F2DD
:10759000BB3201F0CFFA1B4840F2BB3101F0C3FA15
:1075A000EFF3058353B1174914484FF46F7201F09C
:1075B000C1FA14484FF46F7101F0B5FAA268D37B99
:1075C00001330020D373FFF7F5FD0A48FFF78EFB68
:1075D00040B909490948B92201F0ACFA0648B92175
:1075E00001F0A1FA85F31188BFF36F8FBDE8384031
:1075F00002F006B8C80F0020B09F00002F9C0000CA
:107600008C0F00205AA400000B4B994210B50C4679
:107610000AD10A490A4840F23D4201F08BFA074874
:1076200040F23D4101F07FFAD4E9003213605A6024
:107630000023C4E9003310BD500700205AA4000005
:107640002F9C000070B590F90D20437B002A044662
:1076500006DA03F07F03437301461D48FFF7D4FFAA
:10766000637B63F07F0363731A4B9C4208D11A4912
:107670001A48BA2201F05EFA1748BA2101F053FA0B
:10768000174A1146506A51F8203F8B4208BF002329
:1076900023B9C4E90010046054620CE094F90E5060
:1076A00093F90E60B5420ED0AE420CDD5968C4E9C4
:1076B00000310C605C609068031B5842BDE870406C
:1076C0005841FFF777BD9842E3D01B68E0E700BF61
:1076D000AC0F0020500700205AA400002F9C00008F
:1076E0008C0F002070B505464FF02003EFF3118694
:1076F00083F31288BFF36F8F2548FFF7E9FA40B98B
:10770000244925488E2201F015FA22488E2101F0E5
:107710000AFA1F48FFF7FAFA204B214A9C681168C1
:107720008C4214D12046FFF731FD1948FFF7DEFAED
:1077300040B918491848B92201F0FCF91548B92197
:1077400001F0F1F986F31188BFF36F8F70BD00214E
:107750001160144A1268C2B1E2897F2A15D8627B8F
:10776000D20612D1104A94F90E10126891420CDB25
:107770000E4A944209D01A69AA4203DC2046FFF758
:1077800061FFCFE7521B1A61CFE70022FBE700BF82
:10779000C80F0020B09F00002F9C00008C0F00201D
:1077A000BC0F0020C40F0020C00F00205007002095
:1077B00010B590F90D20437B002A044606DA03F049
:1077C0007F03437301460648FFF71EFF054B986889
:1077D000031B5842BDE810405841FFF7EBBC00BF07
:1077E000AC0F00208C0F002038B504460D46FFF783
:1077F000DFFF637B43F00203637345B3144BA56063
:107800009C4208D113491448BA2201F093F9114857
:10781000BA2101F088F92B689D4209D16B68C4E94F
:1078200000531C606C6012E06A689342F6D01B68DB
:10783000002BF3D094F90E2093F90E108A42F3D066
:107840009142F1DD5A68C4E9003214605C6038BDD1
:10785000500700205AA400002F9C00002DE9F041A1
:107860000446884616461D464FF02003EFF3118765
:1078700083F31288BFF36F8F1A48FFF729FA40B9D4
:1078800019491A488E2201F055F917488E2101F046
:107890004AF91448FFF73AFA20464146FFF7A4FF99
:1078A0001048FFF723FA40B90F491048B92201F0F8
:1078B00041F90D48B92101F036F987F31188BFF37A
:1078C0006F8FB5F1FF3F08BFB6F1FF3F08D03246DA
:1078D0002B4604F118000649BDE8F04100F0F2BB68
:1078E000BDE8F081C80F0020B09F00002F9C000071
:1078F0002D7B000038B50E4B054698680D4B0C46A5
:1079000018601146DDE90423FFF7A8FF2846FFF7BA
:10791000EDF940B908490948D02201F00BF90648B1
:10792000D02101F000F92046BDE83840FBF7FEB950
:107930008C0F0020BC0F0020B09F00002F9C000087
:10794000F8B504460E464FF02003EFF3118783F39A
:107950001288BFF36F8F3348FFF7BAF940B9324945
:1079600032488E2201F0E6F82F488E2101F0DBF834
:107970002C48FFF7CBF9637BDA0676B227D1A569ED
:107980002DBB03F07F03637329482146FFF73CFEBC
:10799000637BA67363F07F036373264B9C4208D11D
:1079A00025492248BA2201F0C5F82348BA2101F03E
:1079B000BAF8224A134653F8201F994218BF0D46C1
:1079C000516ACDB9C4E900310C60546221E0A6735C
:1079D00000241448FFF78AF940B913491348B92223
:1079E00001F0A8F81048B92101F09DF887F311883B
:1079F000BFF36F8F2046F8BD94F90E0095F90E6025
:107A0000B0420BD0864209DD6B68C4E900531C60AC
:107A10006C600120FFF7CEFB0124DAE7A942D1D048
:107A20002D68CEE7C80F0020B09F00002F9C0000FB
:107A3000AC0F0020500700205AA400008C0F00203B
:107A400070B50446183000F0EDFB4FF02003EFF363
:107A5000118683F31288BFF36F8F2048FFF738F940
:107A600040B91F491F488E2201F064F81C488E213E
:107A700001F059F81948FFF749F994F90D20637B93
:107A8000002A06DA03F07F03174863732146FFF7E5
:107A9000BBFD164D637BA86843F010036373031BA3
:107AA00058425841FFF786FB0C48FFF71FF940B9D1
:107AB0000B490C48B92201F03DF80948B92101F001
:107AC00032F886F31188BFF36F8FAB68A34203D1FE
:107AD000BDE8704001F094BD70BD00BFC80F00202C
:107AE000B09F00002F9C0000AC0F00208C0F0020E6
:107AF000836810B5044653B90A490B4840F2B922CD
:107B000001F018F8074840F2B92101F00CF8A0681C
:107B10002146FFF779FD637B23F0020363730023A3
:107B2000A36010BD5AA400002F9C000070B504464D
:107B30004FF02003EFF3118683F31288BFF36F8FAA
:107B40001B48FFF7C5F840B91A491B488E2200F0C0
:107B5000F1FF18488E2100F0E6FF1548FFF7D6F830
:107B600014F80B3C13F0280F10D154F8103CA4F17A
:107B7000180513B12846FFF7BBFF14F80B3C23F0A0
:107B8000140304F80B3C2846FFF744FB0848FFF7B2
:107B9000ADF840B907490848B92200F0CBFF0548C5
:107BA000B92100F0C0FF86F31188BFF36F8F70BD5D
:107BB000C80F0020B09F00002F9C000070B5054644
:107BC0004FF02003EFF3118683F31288BFF36F8F1A
:107BD0001748FFF77DF840B9164917488E2200F084
:107BE000A9FF14488E2100F09EFF1148FFF78EF880
:107BF0002C68A5421AD034B12046FFF779FF04F172
:107C0000180000F00FFB0A48FFF770F840B9094967
:107C10000948B92200F08EFF0648B92100F083FF21
:107C200086F31188BFF36F8F204670BD0024EAE70A
:107C3000C80F0020B09F00002F9C0000044B0021C3
:107C400003F12002C3E908220846FFF72BBB00BF5F
:107C50008C0F0020F8B5EFF3058353B1374938484E
:107C600040F2325200F066FF344840F2325100F0E8
:107C70005AFF4FF02003EFF3118683F31288BFF30E
:107C80006F8F3048FFF724F840B92F492C488E22D7
:107C900000F050FF2C488E2100F045FF2B4D294865
:107CA000FFF734F8A9684B7B03F07F034B7305F1B2
:107CB0002000FFF7A9FCAC68637B63F07F0363736C
:107CC000234B9C4208D11D491D48BA2200F032FFC7
:107CD0001A48BA2100F027FF2B6A1E496A6A8B42B4
:107CE00008BF002323B9C4E9001214606C620CE0E1
:107CF00094F90E0093F90E70B8421BD0874219DD3B
:107D00005A68C4E9003214605C600120FFF752FA3F
:107D10000C48FEF7EBFF40B90B490948D02200F0B0
:107D200009FF0948D02100F0FEFE3046BDE8F840CA
:107D3000FAF7FCBF9342D6D01B68D3E75AA40000E1
:107D40002F9C0000C80F0020B09F00008C0F002067
:107D500050070020AC0F00202DE9F04105460E46EB
:107D6000EFF3058353B13849384840F24E5200F0E2
:107D7000E1FE354840F24E5100F0D5FE55EA0603CB
:107D800003D1FFF767FF002058E0AA1C76F1FF330C
:107D900056DB01F03FFC44194FF02003EFF311884C
:107DA00083F31288BFF36F8F2948FEF791FF40B924
:107DB000284926488E2200F0BDFE26488E2100F07C
:107DC000B2FE254F2248FEF7A1FF244BB868186089
:107DD000FFF7EEFCB86822492A463346183000F017
:107DE00071F9BA681A48537B43F010035373FEF7D6
:107DF0007DFF40B917491548D02200F09BFE154879
:107E0000D02100F090FE4046FAF790FFBB685B7B04
:107E1000DB060AD50C490D4840F26F5200F08AFE8D
:107E2000094840F26F5100F07EFE01F0F3FB201A8A
:107E300063EB0303012873F10003A4DBBDE8F081C9
:107E40006FF00104641BA7E75AA400002F9C0000F8
:107E5000C80F0020B09F00008C0F0020BC0F002036
:107E60002D7B000038B505460C46EFF3058353B172
:107E70001149124840F27E5200F05CFE0E4840F27A
:107E80007E5100F050FEB4F1FF3F08BFB5F1FF3F57
:107E900006D10B4B9868FFF7D3FD4FF0FF3038BD8C
:107EA00028462146FFF758FF4FF47A7380FB0303FF
:107EB000C00B40EA4340F2E75AA400002F9C0000A8
:107EC0008C0F0020014B9868704700BF8C0F00207A
:107ED0002DE9F04104464FF02003EFF3118683F3C0
:107EE0001288BFF36F8F3E48FEF7F2FE40B93D495E
:107EF0003D488E2200F01EFE3A488E2100F013FE0F
:107F00003748FEF703FF637B1A0712D53448FEF7A4
:107F1000EDFE40B933493448B92200F00BFE314838
:107F2000B92100F000FE86F31188BFF36F8FBDE822
:107F3000F08123F0200242F00801D20938D16173A8
:107F4000A36813B12046FFF7D3FD04F1180000F039
:107F500069F904F158074FF00008A56DBD4200D043
:107F600085BB0120FFF726F9204B9B68A342CDD1AA
:107F7000EFF30583002BC9D11948FEF7B7FE40B9CE
:107F800018491948D02200F0D5FD1648D02100F03C
:107F9000CAFD3046FAF7CAFE1549134840F2AC62F2
:107FA00000F0C8FD124840F2AC6100F0BCFDADE746
:107FB00003F05F0343F008030E4863732146FFF7A5
:107FC00023FBBDE72846FFF793FD05F1180000F0FD
:107FD00029F9C5F878802846FFF71CF9BDE700BFEE
:107FE000C80F0020B09F00002F9C00008C0F0020C5
:107FF0005AA40000AC0F002008B50648064A0749FD
:10800000121A01F0B7FABDE80840054A05490648CA
:1080100001F0B0BA0000002030070020A0A400004A
:1080200000000000A0A4000000000020034B1B681B
:108030000BB9FCF72BBE0020704700BFCC0F00200F
:10804000114B10B51C689C420AD1FFF7EFFF6FF08F
:1080500000400E4B1B6913B19842A8BF184610BDD3
:10806000FFF7E4FF002CF2D0D4E904321B1A62EBD4
:10807000E072B3F1004F72F10001E8DA002AACBF00
:1080800018460020E5E700BF5C0600208C0F0020AA
:108090000B4A03685268904230B509D043B1D3E926
:1080A0000421D0E90445121941EB0501C3E904217B
:1080B000426813605A600023C0E9003330BD00BF3E
:1080C0005C060020B3F1FF3F08BFB2F1FF3F2DE98E
:1080D000F84304460E4691461D461746984600F062
:1080E0008780036843B148494848632200F022FD75
:1080F0004548632100F017FDA6604FF02003EFF321
:10810000118683F31288BFF36F8F4148FEF7E0FDBD
:1081100040B940493D488E2200F00CFD3D488E217B
:1081200000F001FD3A48FEF7F1FDB9F1FF3F75F1AE
:10813000FF3322DA3849D1E900206FF001039B1A9E
:108140004FF0FF3262EB0000DF1B60EB0800012FF5
:1081500070F1000301DA01270020304AC4E90470FD
:108160001368D2F804C0934208BF002373B9C4E96E
:10817000002CCCF8004054601AE0FFF757FF01379D
:1081800045F100053F1845EBE070E6E7D3E9040749
:10819000D4E90415814275EB070E2BDA401A5968B1
:1081A00067EB0507C3E90407C4E900310C605C60B4
:1081B000136893420BD09C4209D1FFF741FF18B1DD
:1081C000174B1B69834202D00021FCF72DFD10489C
:1081D000FEF78CFD40B90F490C48B92200F0AAFC0B
:1081E0000C48B92100F09FFC86F31188BFF36F8F14
:1081F000BDE8F883091A65EB07056345C4E9041572
:10820000B5D01B68B2E700BF7CA400002F9C000023
:10821000D00F0020B09F0000500800205C06002016
:108220008C0F002038B504464FF02003EFF3118582
:1082300083F31288BFF36F8F1548FEF749FD40B9ED
:10824000144915488E2200F075FC12488E2100F06A
:108250006AFC0F48FEF75AFD2368B3B12046FFF7CA
:1082600017FF00240A48FEF741FD40B909490A48B2
:10827000B92200F05FFC0748B92100F054FC85F3F7
:108280001188BFF36F8F204638BD6FF01504E9E702
:10829000D00F0020B09F00002F9C000038B54FF099
:1082A0002003EFF3118583F31288BFF36F8F134818
:1082B000FEF70EFD40B9124912488E2200F03AFC3A
:1082C0000F488E2100F02FFC0C48FEF71FFDFFF732
:1082D000B7FE04460948FEF709FD40B908490948B8
:1082E000B92200F027FC0648B92100F01CFC85F3F8
:1082F0001188BFF36F8F204638BD00BFD00F00201C
:10830000B09F00002F9C000070B504460D464FF052
:108310002003EFF3118683F31288BFF36F8F1748A2
:10832000FEF7D6FC40B9164916488E2200F002FC32
:1083300013488E2100F0F7FB1048FEF7E7FCFFF72B
:108340007FFE012807DDA04205DBA0422946A8BF29
:108350002046FCF769FC0948FEF7C8FC40B908490B
:108360000848B92200F0E6FB0548B92100F0DBFB24
:1083700086F31188BFF36F8F70BD00BFD00F002050
:10838000B09F00002F9C00002DE9F8430446FFF742
:10839000A9F94FF02003EFF3118583F31288BFF39F
:1083A0006F8F4248FEF794FC40B9414941488E2204
:1083B00000F0C0FB3E488E2100F0B5FB3E4F3B482D
:1083C000DFF8F8803E4EFEF7A1FC3C60D8F8004094
:1083D0003A684445D6E9001E4FEAE2700BD054B12A
:1083E000D4E9043C9A4270EB0C0923DA9B1A6CEB3B
:1083F000000CC4E9043C51184EEB00000024C6E90F
:1084000000103C60FFF71CFE2146FCF70DFC2748DE
:10841000FEF76CFC40B926492648B92200F08AFBD9
:108420002348B92100F07FFB85F31188BFF36F8FDC
:10843000BDE8F88359184EEBE370D31A3B60002275
:108440000023C6E90010C4E904232046FFF720FEFC
:108450001648FEF74BFC40B915491648B92200F002
:1084600069FB1348B92100F05EFB85F31188BFF367
:108470006F8FA368204698474FF02003EFF31185D4
:1084800083F31288BFF36F8F0848FEF721FC40B9D1
:10849000074908488E2200F04DFB05488E2100F068
:1084A00042FB0248FEF732FC90E700BFD00F0020ED
:1084B000B09F00002F9C0000CC0F00205C06002025
:1084C0005008002070B54FF02003EFF3118683F3BE
:1084D0001288BFF36F8F1648FEF7FAFB40B91549B3
:1084E00015488E2200F026FB12488E2100F01BFB5F
:1084F0000F48FEF70BFCFCF7C9FB104AD2E9004518
:1085000004190B4845F10005FEF7F0FB40B9094995
:108510000948B92200F00EFB0648B92100F003FB20
:1085200086F31188BFF36F8F2046294670BD00BFC8
:10853000D00F0020B09F00002F9C000050080020AA
:1085400010B50A4C23681BB101232360002010BD25
:1085500000F0CEF80028F7D00138062803D8044BE5
:1085600053F8200010BD034810BD00BFD40F0020F9
:10857000689B0000FE8FFFFFBFF34F8F0549064B3E
:10858000CA6802F4E0621343CB60BFF34F8F00BFB1
:10859000FDE700BF00ED00E00400FA0510B4094B50
:1085A00009490A4C4FF0FE32C3F800244968C3F869
:1085B0000424C3F80824C3F80C240023C4F80035AD
:1085C00010BC084700B002506406002000A0025012
:1085D000D0E90012014BC3E9001270476406002085
:1085E00010B5044630B16368DB0602D50023236072
:1085F000636010BD024B03485B689847F3E700BF18
:1086000064060020849B0000B0B1436893B1DB0690
:108610000ED5012350E8002F194640E8001C9CF0BD
:10862000000FF7D1012AF5D0BFF35F8F002070470C
:1086300003487047034870476FF4E040704700BF3D
:10864000E98FFFFFEA8FFFFF68B143683BB1DB06AC
:1086500007D5BFF35F8F00230360184670470348B8
:108660007047034870476FF4E0407047EA8FFFFFA0
:10867000E98FFFFF10B5044620B1002211232260CC
:10868000636010BD0148FFF789FFF6E7AC9B00006F
:1086900070B5D0E90023134C134D6360D0E902306C
:1086A000C4E902302260114B0868186048685860BD
:1086B00088689860D1E90301D8601961D5F818314C
:1086C000DB060DD50023C5E94533C5E96E3305F555
:1086D0008A709047236805F5DC70BDE87040184744
:1086E00070BD00BF74060020EC0F0020840600203F
:1086F00038B500F02FF820B1032400F063F82046CD
:1087000038BD00F031F898B900F0ACF898B90F4DC9
:10871000D5F828391B0EF02B08D1D5F8242A0C4B9C
:108720009A420AD0072400F017F8E6E70624FAE791
:108730000424204638BD0024F5E7012000F092F81B
:1087400004460028F7D1C5F80C0AD8E700B002505B
:108750000000E0200020704700207047014BC3F864
:10876000040A704700B0025010B5114800F048F8F4
:1087700000B110BD0F4800F043F80028F9D10E4CAD
:10878000204600F03DF80028F3D10C4B0C481C604B
:1087900000F036F801460028EBD100F02DF8044631
:1087A00008B1204610BD00F03FF82046FAE700BFB0
:1087B000BC060020B0060020B8060020C00600203D
:1087C000B406002008B5084800F024F8074800F077
:1087D00021F8074800F01EF8064800F01BF8BDE835
:1087E000084000F00BB800BFBC060020B006002017
:1087F000B8060020B406002000207047704700BF74
:1088000008B5034B02681B6810689847002008BD34
:108810007406002008B5034B02685B68106898472F
:10882000002008BD7406002070B5094C094D206970
:10883000AB68984718B1084B08485B689847084AE6
:10884000EB68206900211160BDE87040184700BF47
:10885000840600207406002064060020D09B0000DF
:10886000E80F002070B51B4D1B4E0446B268286906
:108870009047F8B95CB1194C2368B3B1012B1BD0F8
:10888000013B23602869F3689847002070BD134CB2
:10889000216841B9124B0122C3F80025114AD2F8D0
:1088A0001039002BFBD101312160F368286998470A
:1088B000002070BD0C4870BD0A4AD2F81039002B58
:1088C000FBD1074A6FF07E40C2F80035FFF746FF44
:1088D0002368D5E78406002074060020E80F0020F6
:1088E00000A0025000B00250E98FFFFF7047062938
:1088F00005D8042912D8032905D0042908D0002856
:1089000008BF822007E000280CBF82202920704782
:10891000002808BF812018BF28207047002814BFF6
:108920002A2084207047002814BF28208220704706
:108930007047D0F8103510B5DBB20C0FC3F1200230
:108940000901A3F12000D94004FA02F2114324FAEC
:1089500000F0084310BD053801288CBF002001201D
:108960007047D8207047082070470F207047034693
:1089700058B1426802F00302012A03D0032A04D14D
:10898000026812B10020986070476FF015007047C0
:10899000002070470FB407B504A951F8040B0191EA
:1089A000F9F782F803B05DF804EB04B07047838BED
:1089B00013F0070305D10368002B0CBF0020032030
:1089C0007047022B05D1C08BB0FA80F040098000BF
:1089D0007047012B05D10368002B0CBF0020052038
:1089E00070470020704710B50C4600B111B96FF008
:1089F000150010BD081DFFF7BAFF0028F9D1A368C4
:108A0000032BF6D9F3E72DE9F0410D460746194649
:108A1000281D90461E46F9F721F8044638B1334622
:108A2000424629463846A446BDE8F0416047BDE8C5
:108A3000F08138B50C46054658B151B10B6843B1C9
:108A40004B6833B12022002100F0D8F82C610020BF
:108A500038BD6FF01500FBE7044608B5084611461F
:108A60001A46A047FFF72EFAFAF7CCFB2DE9F84F8C
:108A70009A46D3786F2B80460F461546A3F1410BDB
:108A800029D024D8582B0CBF10260A26DDF82890B0
:108A90003246002340463946F7F732FB092AD4B262
:108AA0001ED83034B045E4B277F1000709F8014D23
:108AB00001D3D14511D82B789B0605D5082E15D1A9
:108AC000AB7843F00803AB704846BDE8F88F03F07D
:108AD000F703702BD7E70826D8E780460F46D7E77D
:108AE000BBF1190F94BF37345734DBE7102EEBD1AD
:108AF000AB7843F01003E6E72DE9F04107468846DE
:108B000015461E461446B44205D30EB1601B08E05C
:108B10002378002BFAD014F8010B4146B8470028FF
:108B2000F1DABDE8F081404080F311884FF0040095
:108B300002DF70470FB407B504A951F8040B019187
:108B4000F8F7B2FF03B05DF804EB04B0704770476C
:108B500008B50020F9F7FEFDFDF716BE01460068D6
:108B6000FDF712BE00210120FFF7F6BF08B5FAF7A6
:108B7000BDF8BDE80840FAF795B90139034611F888
:108B8000012F0AB91A70704703F8012BF7E7034663
:108B900000201A5C02B970470130FAE70346002052
:108BA0001A5C0AB1884200D170470130F8E7431ED1
:108BB000013913F8012F11F8010F824201D1002A67
:108BC000F7D1101A704710B55AB10139841810F84E
:108BD000012B11F8013FA04201D09A42F7D0D01AE0
:108BE00010BD1046FCE710B5431E0A44914200D167
:108BF00010BD11F8014B03F8014FF7E7C9B2024469
:108C00000346934200D1704703F8011BF9E7062899
:108C100008D14FF080430122C3F80025BFF34F8FE6
:108C200020BFFDE77047002383F31188BFF36F8FE8
:108C300070474FF02003EFF3118283F31288BFF3E4
:108C40006F8F036803F0C00343F00203036082F3F5
:108C50001188BFF36F8F7047F8B5069F0469C9B2DA
:108C60004FF02005EFF3118685F31288BFF36F8F65
:108C70000C2505FB0144A56C05F0070CBCF1010FA8
:108C80000CD1A76486F31188BFF36F8FC4E910235A
:108C9000436853F8313098470020F8BD05F0C0050F
:108CA000AF4286F31188BFF36F8F0CBF6FF0770070
:108CB0004FF0FF30F1E713B580240094FFF7CCFFAD
:108CC00002B010BD0069CBB200EB43100021104789
:108CD0000020FCF71BBA0020FCF776BA8022FAF7D6
:108CE00021BC1046FEF7B2B943685B68D3F8103573
:108CF0000B600020704743685B68D3F8040542406E
:108D00000A404240C3F804250020704743685B686E
:108D10000020C3F80815704743685B680020C3F85B
:108D20000C15704743685A68D2F804354B40C2F8B6
:108D300004350020704730B50B6813B9136018462E
:108D400004E00468656815B12068156030BD08341A
:108D5000013B04600B60EFE738B503680446E3B1FC
:108D60009868D0B10568C5B149B10121FAF78EFF05
:108D700023689B689868BDE8384000F051BC12B980
:108D80009B88DB0409D4806800F04AFC236800213A
:108D90009868BDE83840FAF779BF38BD10B50122B0
:108DA00000210446FFF7D8FFA36933B9636004F1DB
:108DB0001000BDE81040FEF749B910BD0069036816
:108DC0008B4210B506D190F85C4034B9FFF7E6FF4E
:108DD000204610BD6FF01500FBE76FF00F00F8E7BD
:108DE00038B503780C46002B3CD18B6C8D6D93B15C
:108DF0009D4210D85B1B8B6443BB4B6B08334B63AA
:108E00008B6B013B8B6301F1480204F13400383174
:108E1000FFF791FF6064236D9BB19D4211D85B1BEE
:108E20002365CBB9E36B0833E363236C013B236415
:108E300004F1500204F1400104F13C00FFF77BFF14
:108E4000E064606DBDE83840FAF7F4BF4B6C002B6E
:108E5000E1D02B444B64DEE7E36C002BF1D02B44D4
:108E6000E364EEE738BD30B50B6813B913601846FC
:108E700004E00468656815B12068156030BD0834E9
:108E8000013B04600B60EFE738B503680446E3B1CB
:108E90009868D0B10568C5B149B10121FBF736F931
:108EA00023689B689868BDE8384000F0B9BB12B9E8
:108EB0009B88DB0409D4806800F0B2FB23680021A2
:108EC0009868BDE83840FBF721B938BD10B50122DC
:108ED00000210446FFF7D8FFA36933B9636004F1AA
:108EE0001000BDE81040FEF7B1B810BD006903687E
:108EF0008B4210B506D190F85C4034B9FFF7E6FF1D
:108F0000204610BD6FF01500FBE76FF00F00F8E78B
:108F100038B503780C46002B3CD18B6C8D6D93B12A
:108F20009D4210D85B1B8B6443BB4B6B08334B6378
:108F30008B6B013B8B6301F1480204F13400383143
:108F4000FFF791FF6064236D9BB19D4211D85B1BBD
:108F50002365CBB9E36B0833E363236C013B2364E4
:108F600004F1500204F1400104F13C00FFF77BFFE3
:108F7000E064606DBDE83840FBF79CB94B6C002B9A
:108F8000E1D02B444B64DEE7E36C002BF1D02B44A3
:108F9000E364EEE738BD02690B46D2E9010183E8DC
:108FA00003000020704743681B68D3F88004C3F8AF
:108FB00080047047436802691B68D3F8100148B108
:108FC000527C0A700020C3F81001D3F8102101224E
:108FD0001A6070474FF0FF30704702680346D2F8BE
:108FE000580140B95B689B0706D4D2F820010038CD
:108FF00018BF012070470120704742681368D3F8FA
:109000000413C90518D5D3F82011A9B14FF02000D9
:10901000EFF3118180F31288BFF36F8FD3F8200133
:1090200030B10020C3F82001D3F820010120D8601E
:1090300081F31188BFF36F8F5268D20615D54FF0B8
:109040002001EFF3118281F31288BFF36F8FD3F801
:10905000581111B10021C3F800154FF48001C3F875
:10906000081382F31188BFF36F8F70472DE9F34126
:10907000466805693468F7680021C4F80015804621
:10908000286001AA384600F058F8002833DB019B1D
:109090003A681979186800F088F800282BDB291D38
:1090A0004046FBF7A3FA30BB0823C4F80035337AF7
:1090B0005BB9C4F81001D4F8103105F11103C4F8FC
:1090C00034350123C4F83835236073689A075CBFD0
:1090D0004FF48072C4F80423DB0644BF4FF48003CE
:1090E000C4F8043310350023C4F84455C4F8483597
:1090F0000123A360E36002B0BDE8F08110B5002257
:10910000044601212820F9F7C9FD2820F9F796FD2A
:109110002046BDE81040FFF7A9BF10B50022044665
:1091200001210220F9F7BAFD0220F9F787FD204658
:10913000BDE81040FFF79ABF704730B54368136031
:10914000037A03F10053013BDB00456814681D44BA
:10915000AC4202D96FF0010030BD65798D4202D07A
:1091600008341460F1E70020F6E773B500F480538B
:10917000002B044600F03F0301A80BBF1546012554
:109180000E4600260193FBF78BFDC4F3811304F414
:10919000706444EA8304019B344303F5E07344EABA
:1091A000450440F8234002B070BD73B5154604462F
:1091B00000EB8106B44202D1002002B070BD2368EA
:1091C0001A0C062A51D8DFE802F004171D4B223989
:1091D0004B0003F03F03C5F80C35236801A803F0EA
:1091E0003F030193FBF75CFD019B012202FA03F3AD
:1091F000C0F8083511461CE003F03F03C5F81435EC
:109200000022F7E703F03F03C5F80835E5E703F070
:109210003F03C5F80835236801A803F03F03019315
:10922000FBF73EFD019B012101FA03F3C0F80C3569
:1092300000222068FFF799FF0434BBE703F03F03E7
:10924000C5F80C35236801A803F03F030193FBF731
:1092500027FD019B012202FA03F3C0F80C35C9E790
:1092600003F03F03C5F81035CAE76FF08500A4E7A7
:1092700008B50020FAF7FEF8FFF762B908B5F9F76C
:10928000F5FBF9F7A7FCBDE80840FFF759B900471F
:1092900000F0C6B943090BD0012B4FF6FF7318BF7E
:1092A000002300F01F0023FA00F000F001007047D7
:1092B0004FF0FF33F5E708B50246FBF7EBFF10B1BF
:1092C0001046FBF7D1FF00F0010008BD2DE9F34186
:1092D000019001A8DDE908580C4617461E46FCF728
:1092E00001F8019B391E18BF012100EB8300231EEA
:1092F00018BF0123002E43EA410314BF0C210021B3
:10930000002D43EA010314BF4FF4E0610021B8F1DE
:10931000000F43EA0103D0F8002714BF4FF4403197
:1093200000210B4322EA030304B124780FB13F78F4
:109330007F001C430EB13678B6003C438DB12978CE
:1093400009023443B8F1000F03D098F800804FEAC7
:109350000848214341EA0801C0F8001702B0BDE8FF
:10936000F0812946EDE71FB50DF10F0301930023AE
:109370008DF80F1000931A461946FFF7A7FF05B0A6
:109380005DF804FB37B5D0F818358A69DBB28DF883
:1093900007300B6A93423EBF4A699DF80740D45498
:1093A0000B6A91F824500C695A1C0A62023335B1D9
:1093B000A3428C6938BF0B619C4288BF8B610D69E9
:1093C0009D4205D9CA68D35CC0F81C3501200AE06B
:1093D0008C699C4201D9CB7FF6E7AA42F6D3A24220
:1093E0002CBF0020012003B030BD07B5019001A8BB
:1093F000FCF728FB019B03F5E073022240F82320D1
:1094000003B05DF804FB07B5019001A8FCF71AFB57
:10941000019A01239340C0F80C3503B05DF804FBBA
:1094200007B5019001A8FCF70DFB019A01239340B9
:10943000C0F8083503B05DF804FB07B5019001A83A
:10944000FCF728FD019A01239340C0F80C3503B0C6
:109450005DF804FB07B5019001A8FCF71BFD019A1C
:1094600001239340C0F8083503B05DF804FB837F07
:109470005A070BD4C07FFF2808D09B0758BF81F044
:10948000010109B9FFF7D9BFFFF7E4BF7047431CDB
:1094900007B509D0019001A8FCF7FCFC019B03F57E
:1094A000E073022240F8232003B05DF804FB2DE9AD
:1094B000F047002406460F46904600F5A0754FF48D
:1094C0008039A2462B687BB1D6F8043309FA04F23E
:1094D0001A4209D0A000C5F800A02B6800F5A073BF
:1094E00098B2D7E9003198470134444505F10405A5
:1094F000E8D1BDE8F08730B54FF4803400688C4087
:1095000063B18B0003F5A0730025C550C358C0F8A4
:10951000044301F5A87140F8212030BDC0F808438C
:10952000F7E770B4046840F20116D4F800528E4098
:1095300025EA0605C4F80052D4F800522B43C4F8BB
:1095400000329DF80C3070BCFFF7D5BFFDF79CB81A
:1095500008B5FFF7FBFF002008BD704738B1C368AE
:109560001888C0F30800A0F580735842584170472E
:10957000FFF744BBFFF737BB30B50024C4618460FC
:1095800041EA020414F00304C0E9033241610CD142
:109590002546A342856103D1C0E90000002030BD0B
:1095A0000D6001340D461144F3E76FF01500F6E746
:1095B000EFF30580003818BF0120704708B5F9F7B0
:1095C00045F9BDE80840FFF7B7BD90F90E308B4272
:1095D00001D0FEF7B5B90020704703460020C3E96B
:1095E0000200C3E900337047034620B9EFF3058258
:1095F0000AB9F9F79BBB83F31188BFF36F8F7047EC
:109600004FF02003EFF3118083F31288BFF36F8FC5
:10961000FFF7EABF08B5FEF755FF08BDFEF752BFDA
:1096200008B1F9F73DBF704770470000FBF78EBBEC
:08963000046BFF7F0100000044
:109638004D34000000000000C9350000A896000065
:1096480051950000000000006D6900000000000056
:10965800913A0000C0960000913A0000D8960000A8
:109668007992000000000000FD900000F0960000D4
:109678001B91000008970000C54A00000000000088
:109688007D92000000000000013D000020970000CE
:109698008141000038970000C50A00000000000062
:1096A80052A10000CC990000DC990000C4060020FB
:1096B800E40D0020F8980000B8A10000F49900001B
:1096C800149A0000C8060020400E0020F2980000FE
:1096D800BFA10000049A0000149A0000CC060020E4
:1096E8004C0E0020EA980000CCA10000E49A00008B
:1096F8003C9B0000D8060020B0050020E49800003C
:10970800D3A10000109B00003C9B0000DC06002059
:10971800C4050020DE980000C6A10000389A0000A9
:10972800809A0000D0060020E8040020D8980000A5
:10973800A09C0000889A0000DC9A0000D406002053
:0897480048050020D098000044
:10975000015200008F92000000000000CD0F0000B9
:1097600008970000FB8F0000315E00008F92000020
:1097700000000000658B000000000000658B000009
:10978000795800008F92000000000000658B0000F7
:10979000000000004D66000000000000616600004F
:1097A00000000000658B000000000000658B0000D9
:1097B00000000000658B000000000000658B0000C9
:1097C00000000000658B000000000000658B0000B9
:1097D00000000000658B000000000000454B000009
:1097E00000000000658B000000000000658B000099
:1097F00000000000658B000000000000658B000089
:1098000000000000658B000000000000658B000078
:1098100000000000658B000000000000658B000068
:10982000000000007566000000000000658B00006D
:1098300000000000658B000000000000658B000048
:1098400000000000658B000000000000658B000038
:1098500000000000658B000000000000658B000028
:1098600000000000658B000000000000658B000018
:1098700000000000658B000000000000658B000008
:1098800000000000658B000000000000658B0000F8
:10989000F0960000FB8F000000000000658B0000C8
:1098A00000000000658B000000000000658B0000D8
:1098B00000000000658B000000000000658B0000C8
:1098C00000000000658B0000C16300008F92000063
:1098D000030000800080FF7F00800080FF7F008009
:1098E0000080FF7F00800080FF7F008000800700F5
:0E98F000FF7F00800080FF7F00800080FF7FF0
:0298FE00FFFF6A
:109900000338FDD8704700001908000079080000EE
:1099100019060000D506000051090000690A000080
:10992000C1080000B10600002D0A0000D8000000A8
:10993000E2000000EC000000F0000000F400000075
:10994000F8000000FC000000000000000200000021
:1099500003000000040000000500000006000000F5
:10996000070000000800000000000000518B00000C
:10997000E0040020D8040020D004002000000000F3
:10998000C8040020652B0000792A0000C12A0000CD
:10999000192B0000000000200000000000000B0652
:1099A00002000000A89900000000000006A10000CD
:1099B00026000207000000200EA1000022000B116B
:1099C000B5340000A135000000000000AD360000F5
:1099D00045370000D18C0000D78C00001137000003
:1099E000DD8C0000B78C000000000000F1340000A6
:1099F00000000000FFFF0000000300500000000016
:109A000001000000FFFFFFFF000000500000000009
:109A100000000000453B0000E98C0000F78C0000CE
:109A20000D8D0000198D0000258D000049390000C2
:109A3000BD380000000000000030004000000000C1
:109A4000000000FF00FF0000000000000000000117
:109A500001000000589A000000300040649A0000A5
:109A6000010000006C9A0000030000001B000400CD
:109A70001A0005001D0006000000000000000000A4
:109A8000B53E0000BD8D000000F002400000000067
:109A9000FFFF00000048E801000000FF0000FF0099
:109AA00000000000000000FF0200000101000000B3
:109AB000B49A000000F00240C09A000001000000CB
:109AC000C89A0000030000000C0004000E0006000D
:109AD0000D000500D89600000F0001006143000052
:109AE000ED8E000000800240000000000000000039
:109AF000F49A000000800240009B0000010000007A
:109B0000089B00000200000004000000C5000100E6
:109B1000002000400000000000000000209B00002A
:109B2000002000402C9B000001000000349B00003E
:109B30000200000016000000D1000100B58F0000F7
:109B400051470000A78F0000ED450000978F0000EF
:109B5000389600008096000088960000A0960000CD
:109B6000A8960000F5FFFFFFFF8FFFFFFF8FFFFFAD
:109B7000FE8FFFFFFE8FFFFFFD8FFFFFFC8FFFFFBC
:109B8000FC8FFFFF6D757465785F66726565206395
:109B9000616C6C65642077697468204E554C4C206C
:109BA000706172616D6574657200000043616E27BB
:109BB0007420696E697469616C697A65206D757469
:109BC00065782C20776173204E554C4C0D0A0000AF
:109BD000436F756C64206E6F74206C6F636B2070C4
:109BE0006F7765722073617665206D757465780096
:109BF00050000000000000005800D002CE01574580
:109C000053545F544F504449522F7A6570687972AB
:109C10002F696E636C7564652F7A65706879722F31
:109C2000647269766572732F6770696F2E68004180
:109C30005353455254494F4E204641494C204020F1
:109C400025733A25640A00574553545F544F5044D6
:109C500049522F6D6F64756C65732F68616C2F6E40
:109C60006F726469632F6E7266782F68616C2F6EF5
:109C700072665F6770696F74652E6800434D414B73
:109C8000455F534F555243455F4449522F737263AA
:109C90002F66656D2F6E726632313534302E63005B
:109CA0005350495F33005374617274696E67204486
:109CB00069726563742054657374204D6F64652008
:109CC0006578616D706C650A005541525420646579
:109CD00076696365206E6F742072656164790A002D
:109CE0004572726F7220647572696E672044544DBC
:109CF00020696E697469616C697A6174696F6E3A22
:109D00002025640A005541525420706F6C6C696EB6
:109D100067206572726F723A2025640A0053656E7F
:109D200064696E67203078253034582044544D20C3
:109D3000636F6D6D616E640A005265636569766577
:109D400064203078253034582044544D20657665A1
:109D50006E740A00496E636F727265637420736576
:109D60007474696E677320666F7220726164696FC4
:109D7000206D6F646520616E6420545820706F7789
:109D800065720A00574553545F544F504449522F4F
:109D90006D6F64756C65732F68616C2F6E6F726484
:109DA00069632F6E7266782F68616C2F6E72665FC2
:109DB000726164696F2E6800556E61626C65207413
:109DC0006F206765742074686520436C6F636B2037
:109DD0006D616E616765720A00436C6F636B207220
:109DE000657175657374206661696C65643A2025D8
:109DF000640A00436C6F636B20636F756C64206E44
:109E00006F7420626520737461727465643A2025F2
:109E1000640A006E7266785F74696D65725F696E60
:109E20006974206661696C656420776974683A209A
:109E300025640A00677070695F6368616E6E656CA7
:109E40005F616C6C6F63206661696C656420776923
:109E500074683A2025640A0044544D20776169747F
:109E6000206572726F723A2025640A00FFC1FBE818
:109E70004C90728BE7B3518963AB23230284187231
:109E8000AA612F3B51A8E53749FBC9CA0C18532CCE
:109E9000FD45E39AE6F15DB0B61BB4BE2A50EAE98F
:109EA0000E9C4B5E5724CCA1B759B887FFE07D7458
:109EB0002648B9C5F3D9A8C4B1D5911101420C39CE
:109EC000D5B0979D28D4F29BA4FD6465068C299695
:109ED000FEA2714DF3F82E58DB0D5A5F1528F5746C
:109EE00007CE25AF2B12E6D0DB2CDCC37FF03E3A49
:109EF00013A4DCE2F96C54E2D8EAC8880021869CFD
:109F00006AD8CB4E146AF94DD27EB23203C6144BD6
:109F10007FD1B8A6797C17ACED06ADAF0A947ABABA
:109F200003E792D7150973E86D16EEE13F781F9DA0
:109F300009526EF17C362A716C7564448010434E70
:109F400035EC65270AB5FC26693F599901638AA556
:109F5000BF685CD33CBE0BD67683D657054A3DDD41
:109F60008173C9EB8A8439F4360BF7574553545F34
:109F7000544F504449522F7A65706879722F6C693A
:109F8000622F6F732F6E6F746966792E6300574569
:109F900053545F544F504449522F7A657068797218
:109FA0002F6C69622F6F732F6F6E6F66662E630062
:109FB000574553545F544F504449522F7A65706847
:109FC00079722F696E636C7564652F7A6570687934
:109FD000722F7370696E6C6F636B2E6800286E69E8
:109FE0006C29004661696C656420746F207265623B
:109FF0006F6F743A207370696E6E696E6720656E5C
:10A00000646C6573736C792E2E2E0A006D75746501
:10A01000785F696E69742063616C6C656420776930
:10A020007468204E554C4C20706172616D6574658A
:10A030007200436F756C64206E6F7420616C6C6F7E
:10A0400063617465206D75746578206265666F72F2
:10A050006520696E697469616C697A696E67005719
:10A060004553545F544F504449522F7A6570687974
:10A07000722F617263682F61726D2F636F72652F2B
:10A08000616172636833322F6972715F6D616E61F5
:10A0900067652E6300574553545F544F50444952EF
:10A0A0002F7A65706879722F617263682F61726DA3
:10A0B0002F636F72652F616172636833322F636F34
:10A0C000727465785F6D2F6661756C742E630057CE
:10A0D0004553545F544F504449522F7A6570687904
:10A0E000722F617263682F61726D2F636F72652FBB
:10A0F000616172636833322F6D70752F61726D5FAD
:10A100006D70752E6300464C4153485F30005352CA
:10A11000414D5F3000574553545F544F50444952AE
:10A120002F7A65706879722F647269766572732F01
:10A13000636C6F636B5F636F6E74726F6C2F636CB5
:10A140006F636B5F636F6E74726F6C5F6E72662E9F
:10A150006300434C4F434B00574553545F544F509B
:10A160004449522F7A65706879722F6472697665F6
:10A1700072732F6770696F2F6770696F5F7574698D
:10A180006C732E6800574553545F544F50444952E6
:10A190002F6D6F64756C65732F68616C2F6E6F72B5
:10A1A0006469632F6E7266782F68616C2F6E7266B9
:10A1B0005F6770696F2E68004750494F5F310047F5
:10A1C00050494F5F30005350495F30005541525461
:10A1D0005F3100554152545F300000000000000123
:10A1E000010000000000574553545F544F5044494C
:10A1F000522F6D6F64756C65732F68616C2F6E6F75
:10A20000726469632F6E7266782F64726976657204
:10A21000732F7372632F6E7266785F636C6F636BFC
:10A220002E6300574553545F544F504449522F6D8D
:10A230006F64756C65732F68616C2F6E6F726469E3
:10A24000632F6E7266782F68616C2F6E72665F6323
:10A250006C6F636B2E6800574553545F544F5044E6
:10A2600049522F6D6F64756C65732F68616C2F6E2A
:10A270006F726469632F6E7266782F647269766597
:10A2800072732F7372632F6E7266785F6770696F77
:10A2900074652E6300574553545F544F50444952E0
:10A2A0002F6D6F64756C65732F68616C2F6E6F72A4
:10A2B0006469632F6E7266782F6472697665727353
:10A2C0002F7372632F6E7266785F7370692E6300EE
:10A2D000574553545F544F504449522F6D6F647526
:10A2E0006C65732F68616C2F6E6F726469632F6E7B
:10A2F0007266782F647269766572732F7372632F3A
:10A300006E7266785F7370696D2E630057455354A3
:10A310005F544F504449522F6D6F64756C65732FB5
:10A3200068616C2F6E6F726469632F6E7266782F2E
:10A33000647269766572732F7372632F6E726678BA
:10A340005F74696D65722E63005465726D696E612C
:10A350006C005254540053454747455200574553EB
:10A36000545F544F504449522F7A65706879722F68
:10A370006B65726E656C2F666174616C2E63006D27
:10A3800061696E00574553545F544F504449522FF2
:10A390007A65706879722F6B65726E656C2F6D656A
:10A3A0006D5F736C61622E6300574553545F544F69
:10A3B000504449522F7A65706879722F6B65726EBE
:10A3C000656C2F7468726561642E63005745535441
:10A3D0005F544F504449522F7A65706879722F6BE1
:10A3E00065726E656C2F69646C652E63005745530A
:10A3F000545F544F504449522F7A65706879722FD8
:10A400006B65726E656C2F6D757465782E63005781
:10A410004553545F544F504449522F7A65706879C0
:10A42000722F6B65726E656C2F696E636C756465F7
:10A430002F6B73636865642E6800574553545F54EF
:10A440004F504449522F7A65706879722F6B65724C
:10A450006E656C2F73656D2E6300574553545F54C2
:10A460004F504449522F7A65706879722F6B65722C
:10A470006E656C2F73636865642E63005745535493
:10A480005F544F504449522F7A65706879722F6B30
:10A4900065726E656C2F74696D656F75742E6300DF
:10A4A0000000000000127A0000010000000000001F
:10A4B000D89600000F00010000000000000000001E
:10A4C000000000000000000000000000D89600001E
:10A4D00008000000D896000007000000C0960000A9
:10A4E00009000000D89600000600000000000000EF
:10A4F00000A0004002040000000000000000000076
:10A50000000000000000000000000000000000004B
:10A51000000000000000000000000000000000003B
:10A52000000000000000000000000000000000002B
:10A53000000000000000000000000000000000001B
:10A710000000000000000000294176710080004028
:10A720000004000000900040010400008C020020A2
:10A730008C020020000000000100000000A0014089
:10A7400003060000000003000000000000000000FD
:10A7500000000000000000000000000000000000F9
:10A7600000000000000000000000000000000000E9
:10A7700000000000000000000000000000000000D9
:10A7800000000000000000000000000000000000C9
:10A7900000000000000000000000000000000000B9
:10A7A00000000000000000000000000000000000A9
:10A7B0000000000000000000000000000000000099
:10A7C0000000000000000000000000000000000089
:10A7D0000000000000000000000000000000000079
:10A7E0000000000000000000000000000000000069
:10A7F0000000000000000000000000000000000059
:10A800000000000000000000000000000000000048
:10A810000000000000000000000000000000000038
:10A820000000000000000000000000000000000028
:10A830000000000000000000000000000000000018
:10A840000000000000000000000000000000000008
:10A8500000000000000000000000000000000000F8
:10A8600000000000000000000000000000000000E8
:10A8700000000000000000000000000000000000D8
:10A8800000000000000000000000000000000000C8
:10A8900000000000000000000000000000000000B8
:10A8A00000000000000000000000000000000000A8
:10A8B0000000000000000000000000000000000098
:10A8C0000000000000000000000000000000000088
:10A8D0000000000000000000000000000000000078
:10A8E0000000000000000000000000000000000068
:10A8F0000000000000000000000000000000000058
:10A900000000000000000000000000000000000047
:10A910000000000000000000000000000000000037
:10A920000000000000000000000000000000000027
:10A930000000000000000000000000000000000017
:10A940000000000000000000000000000000000007
:10A950000000000000000000FF00000000000000F8
:10A9600091890000FFFFFFFFF406002001000000B6
:10A970000807002001000000E006002001000000A0
:10A980001C07002001000000000000000000000083
:10A99000789A000000000000F8040020F80400206D
:10A9A000000000000100000008050020080500204C
:10A9B0000000000001000000000000000000000096
:10A9C0000000000000000000000000000000000087
:10A9D00000000000000000000000000020970000C0
:10A9E0000000000000000000000000000000000067
:10A9F000D49A0000010000005805002058050020EE
:10AA0000000000000100000068050020680500202B
:10AA10000000000001000000000000000000000035
:10AA20000000000000000000000000000000000026
:10AA30000000000000000000000000003897000047
:10AA40000000000000000000000000000000000006
:10AA50000000000000E10000000103000000000011
:10AA60000000000000000000004B00000001030097
:10AA700000000000000000000090D0030000000073
:10AA800000000000000000000000000000000000C6
:10AA900000000000000000000000000000000000B6
:10AAA00000000000000000000000000000000000A6
:10AAB0000000000000000000000000000000000096
:10AAC0000000000000000000000000000000000086
:10AAD0000000000000000000000000000000000076
:10AAE000000000000000000000000000FF00000067
:10AAF0000000000000000000FFFF0F005C060020C7
:10AB00005C0600200000000079850000D80F0020BE
:10AB10001100000075860000E18500000986000034
:10AB200049860000A80600206C060020A006002030
:10AB30000000000098060020DC0F0020110000003B
:10AB4000E00F002011000000E40F002011000000C1
:10AB500088060020940600208C0600208406002031
:04AB6000B806002013
:10AB640000000000000000000000000000000000E1
:0CAB7400000000000000000000000000D5
:10AB8000E0060020E00600200000000000000000B9
:10AB90000E000000F4060020F40600200000000073
:10ABA000000000000E000000080700200807002039
:10ABB00000000000000000000E0000001C07002044
:10ABC0001C07002000000000000000000E00000034
:04000003000031299F
:00000001FF
